:020000040800F2
:10500000D81B0020D5500008858B00084982000875
:105010000000000000000000000000000000000090
:105020000000000000000000000000001D990008C2
:105030000000000000000000CD910008359A000833
:10504000E7500008E7500008E7500008E750000864
:10505000E7500008895D0008E7500008E7500008A5
:1050600000000000E7500008B15C0008E7500008AD
:10507000E75000087587000800000000E7500008AE
:1050800000000000E75000080000000000000000E1
:10509000E750000800000000E7500008E750000853
:1050A000E7500008E7500008E7500008E1A40008B6
:1050B000E7500008E7500008000000000000000072
:1050C0000348854600F040FD0048004761B80008ED
:1050D000D81B00200448804704480047FEE7FEE74D
:1050E000FEE7FEE7FEE7FEE7D19A0008C1500008A0
:1050F00030B50B46014600202022012409E00D4670
:10510000D5409D4205D31D469540491B25469540F7
:1051100040191546521E002DF1DC30BDF0B51FB40C
:105120000646002082B005464024019100901BE015
:10513000019922460F46304600F0F0FB049A059B89
:10514000801A994110D310461946224600F0D6FB2A
:10515000361A8F410197224601200021009F00F05E
:10516000CDFB38184D4100902046641E0028DFDC3E
:10517000019B00982946324607B0F0BD03460B4319
:105180009B0703D009E008C9121F08C0042AFAD2FD
:1051900003E00B780370401C491C521EF9D2704783
:1051A000D2B201E00270401C491EFBD270470022BF
:1051B000F6E710B513460A4604461946FFF7F0FF16
:1051C000204610BD30B504460020034600E05B1CBD
:1051D000934203D2E05CCD5C401BF8D030BDF8B503
:1051E00002464A40D40F42004B0052085B089A42E4
:1051F00002D20246084611464A0023D0C30D4A0097
:10520000DDB2120EAD1A202D35DA49020126490A07
:10521000F6058A19002C00D0524220214F1B11465E
:10522000B9402A411018C20D9A4221D0002C17D043
:10523000012D08DCDA05801AD20F8019D207DBB203
:1052400000F098FBF8BDDA05801A012340001B0628
:10525000C01880185A428018CA0F1043490007E04E
:105260004908C2071143DA05801A801940088018DE
:1052700000F078FBF8BD61000122511A001BF7E72E
:105280000122D2075140AAE70122D2075040A6E7E7
:10529000024670B54A40D30FDB0740002DD04A00CC
:1052A0002AD0010E140E000212020919400A520AF5
:1052B0008418E50104465443000A120A2E045043A0
:1052C000A4194219200CC543AA18120C0125AD03DC
:1052D000521C521912047F39240400D0521C10436E
:1052E00001D44000491EC2B20C06C0092018401C5F
:1052F0004008802A02D003E0002070BD4008400032
:10530000002900DA0020184370BD70B502464A40FB
:10531000D50F40004A00ED0740085208002814D07D
:10532000002A12D0C40DD30D41020120C005520243
:10533000490A520AE41A091812187D34914201D31D
:10534000641C00E04900002C01DA002070BD00233D
:10535000914201D3891A0343400849000028F7D13C
:1053600000290AD0914202D10121C90705E09142EA
:1053700001D2012101E00121C943E005C018401913
:1053800000F0F0FA70BD420005D04200120E524209
:105390008A4201DB00207047C905081870470000E9
:1053A000F0B507460846584087B0C00F0490480043
:1053B0000E46590040084908BC1A884105D23846B3
:1053C00031461E4617460B46024658004008104319
:1053D0004CD0300D039040055900400D490D05900B
:1053E000401A0290402872DA18030121000B0905C7
:1053F0000843019004980092002805D00199524278
:105400000020884100920190029840210A1A0199D7
:10541000009800F073FA05460C466B4607CB00F087
:105420008EFAC0197141039A0E0D0023D71756400A
:105430001A467A40164344D0049A002A2DD0029A84
:10544000012A039A15DC1205C01A9141012636057E
:10545000001C7141D20F059ED20700930192029663
:105460002A46234600F0CCFA07B0F0BD3846314654
:10547000FAE71605224A0F46B218C01AB7410121B1
:105480000905001C4F4100187F4111461818794149
:10549000E20F10436D19644113E0E2076D081543F4
:1054A0006408C2071443039A01261205C01A9141E9
:1054B0003605001C7141CE07400830434908C0182A
:1054C00051412A46234600F08EFACDE7FFE70498C3
:1054D00001224000C117121A00238B410498314663
:1054E000C417381AA141EEE730B40124E407634041
:1054F00030BC55E730B40124E407614030BC4FE7CD
:105500000000E0FFF0B51FB488B00B9909980024A3
:1055100048400999C00F490049080991C0070B99F3
:105520000090490049080B9109990898A64608433C
:105530001CD00B990A98084318D009980124400000
:10554000420D4800410D099824050003000B20433B
:1055500009900B980003000B20430B9050181C4936
:105560004018002201901446104605E00020014634
:105570000DB0F0BD032801DA034600E003239C468A
:10558000C11A0AAE0AE05F0008ADED5B4F00F75BA1
:105590007D430027AA187C41491C5B1E6145F2DD52
:1055A000410004AB5A522104120C0A43240C401C43
:1055B0000828DFDB01980290009970460191009065
:1055C000059B049A0799069800F01AFAD0E70000A4
:1055D0000DFCFFFFF0B50C465C4085B0E40FE4071E
:1055E00003944C000026640859009446490802467A
:1055F0000296224321D062460A431ED06200570D14
:105600004A000E032303550D012402462C492405AC
:10561000781B1B0B360B4018234326436146009032
:105620001C46501AB44103D30098401C009002E07D
:10563000921800985B41002803DA0020014605B06B
:10564000F0BD0020012109050746864611E06446A9
:105650001D46141BB54106D36546521BB341744623
:1056600007430C43A646CD07400849082843921833
:105670005B4105460D43EAD11046184313D06046FE
:10568000194650407140084306D06046101AB34195
:1056900006D20122002306E000220123DB0702E0FC
:1056A0000122D2435310009874460105381C614111
:1056B000029C039D0019694100F095F9BFE70000C5
:1056C000FD03000070B54B005B0803430BD04B009B
:1056D0005C0D002633466542B341D417AD1AA34191
:1056E00002DB0020014670BD12053018514170BD2B
:1056F000C217C10F504010B54018CA0796230021A9
:1057000000F038F910BD10B500229623114600F0C4
:1057100031F910BD0EB5C217C10F5040CA0740186D
:105720000021054B0293019200910A460B4600F0BE
:1057300067F903B000BD0000330400000EB5054951
:105740000291002100910A460B46019100F058F9A0
:1057500003B000BD33040000C20F4100400201232A
:10576000400ADB05D207090EC0187F2901DA0020A4
:105770007047962903DC9623591AC84001E09639F0
:105780008840002AF4D04042704741004002012284
:10579000400AD205090E80187F2901DA00207047DF
:1057A000962903DC9622511AC840704796398840E2
:1057B0007047000070B5CD0F4A0009030123090BA3
:1057C0001B0519430B4BED070024520D9A4201DAD9
:1057D000002070BD074B34339A4203DC9A1A00F064
:1057E0009DF802E00449511888402C43F1D0404212
:1057F00070BD0000FF030000CDFBFFFF4A0009035E
:105800000123090B1B051943094B10B5520D9A4290
:1058100001DA002010BD064B34339A4203DC9A1A99
:1058200000F07CF810BD03495118884010BD0000FD
:10583000FF030000CDFBFFFFC20FD207400040086E
:105840000BD0C10D0723DB01C91840020905400A2E
:105850001143C208400711437047002001467047BA
:1058600010B5002904DB0124E40740428C412146A5
:10587000002B04DB1C460123DB075242A3418B4271
:1058800000D1824210BD000010B5002904DB0124C4
:10589000E40740428C412146002B04DB1C460123D7
:1058A000DB075242A341994200D1904210BD000053
:1058B000CB0FDB07490010B5490802460A4307D061
:1058C0000A0D07240903E401090B121B002A01DC5D
:1058D000002010BDC900440F0C43C100E018D205E0
:1058E000801800F03FF810BD0122D207002800DB2D
:1058F000101A002900DB511A8142704710B5202A86
:1059000004DB0146203A9140002010BD9140202345
:105910009C1A0346E3401943904010BD10B5202A5D
:1059200004DB0846203AD040002110BD0B46D3408E
:10593000D0402024A21A91400843194610BD10B54A
:10594000202A06DBCB170846203A1041C1170B432B
:1059500006E00B461341D0402024A21A9140084390
:10596000194610BD002904DA401C490001D1400845
:105970004000704770B40024050C05D110240004C9
:1059800002D1002921D01124050E01D100020834D2
:10599000050F01D10001241D850F01D18000A41C39
:1059A000002801DB4000641C002908D020252E1BA4
:1059B0000D46F540A14000D00121294308430106CE
:1059C0001B1B000ADB1D02D5002070BC7047DB05E5
:1059D000181880180029F8DA401C4900F5D170BC6D
:1059E00040084000704710B5002B08DA0024401C26
:1059F000614192185B411A4301D14008400010BD3B
:105A0000F0B51FB482B005460C0003D0084604F080
:105A100021FE02E004F01EFE2030024600902146E6
:105A20002846FFF76BFF049B059A04460F46184370
:105A30001143084314D0184610431BD0009840214E
:105A40000A1A18460599FFF769FF05460E46009A9F
:105A500005990498FFF752FF084305D0012004E0A0
:105A60002046394607B0F0BD0020C11705430E435C
:105A70002C43374300990E986305401A7905E40AD0
:105A800000220C43FD0A0A3002D500200146E9E756
:105A90000105101969410C9C0D9D00196941FFF722
:105AA000A2FFDFE7FEB500231A461B1A8A4103DB7B
:105AB0000020014603B0F0BD4A000D0301212D0B6B
:105AC0000905520D0D43D10702D100186D41521E38
:105AD0005110FF31FF310131002704463E46384660
:105AE000009701910246012100200905FFF716FFEA
:105AF000C3197141F818324684468E464A416146C0
:105B00002846611A904104D36046241A954176468E
:105B10001F46241900986D41401C00903428E1DD97
:105B2000F91930467041091BA84103D20022D24323
:105B3000134601E00022134601980105381C71410B
:105B4000FFF751FFB6E70000064C0125064E05E0C1
:105B5000E36807CC2B430C3C98471034B442F7D38E
:105B6000FFF7B2FAB0C60008D0C6000870B58C18AE
:105B70000578401C6B075B0F01D10378401C2A118C
:105B800006D10278401C03E006780E70401C491CC8
:105B90005B1EF9D12B0705D40023521E0DD40B70C8
:105BA000491CFAE70378401CCB1A921C03E01D78CD
:105BB0000D70491C5B1C521EF9D5A142D8D30020A0
:105BC00070BD000038B50446064805490068FFF777
:105BD0008FFA604300E0401E00900028FBD138BDE2
:105BE00040420F007C010020F8B50446006881683F
:105BF0008907890F012902D10168C90722D181686B
:105C0000114A10261140012500290ED1816829432F
:105C100081600120FFF7D6FF01F010F807460CE085
:105C200001F00CF8C01B0A2807D9606D304360658D
:105C3000A06D2843A0650120F8BD20680068C0431E
:105C4000C007EDD10020F8BD170000801FB50B483C
:105C500000900B4801900B4802900B480390694656
:105C60000A4805F0EDF80A4A08481146083904F0D8
:105C7000D5FF00F057FA002004B010BDB9C40008E9
:105C800095C40008F5C40008F3C40008880100208A
:105C90001000002010B500231A4603E0845CE318CE
:105CA0009BB2521C8A42F9D3D84380B210BD000087
:105CB00010B5034800F07EFD024800F07BFD10BDEA
:105CC000781700203017002030B5446C1C252C407C
:105CD0000125A540046C6560046863608368102B2F
:105CE000036803D099600068C26030BD9A600068A4
:105CF000C16030BD1449012048720A4602205E325C
:105D0000507203203C3A507204200E3A50720F48F1
:105D10000D4B0078087022310870203108770C494B
:105D20005A1C087858714978997123331871597140
:105D3000203318775977107551751A461E32107531
:105D40005175107651767047E01100202701002030
:105D50004C01002010B503F0B7FD202003F060FED9
:105D6000012005F0D7FA002003F05AFE044805F0A0
:105D700075F9044805F024FC002005F059FC10BD1D
:105D8000E800002083800000F8B50520012100070D
:105D900000F040FF0025174C002800D06560164E2B
:105DA0000221304600F036FF00281BD10120207070
:105DB0001248808F00280ED00127BF0200223946EA
:105DC000304600F034FF0A2004F098FE01223946E4
:105DD000304600F02CFF0A48656000880A214843DD
:105DE00008490880012000F04DFE022000F04AFE24
:105DF000F8BD00006801002000040050E00D002004
:105E000034010020480100207047000010B5084907
:105E100000224A6107494B684C1523434B604B688D
:105E2000082423434B60C009C001026010BD00007C
:105E3000C0170020002002407FB500250C46064612
:105E4000039500F0EFFDE009029003A9019600958B
:105E5000684600F07FFD002804D000F0B7FD002068
:105E600004B070BD00F0B2FD0120F9E710B50023C9
:105E700002E0C45CCC545B1C9342FAD310BD00001A
:105E800010B5214A00219069C305204804D5416915
:105E9000022319434161911593699B0505D5436917
:105EA0000124234343616302194393695B0505D5CC
:105EB0004369082423434361E301194393691B05A4
:105EC00005D543690424234343616302194393695D
:105ED0009B0405D54369102423434361630219439E
:105EE00093699B0304D5446920231C4344611943EF
:105EF0009369DB0305D54369402423434361A00232
:105F00000143916110BD000000200240C017002035
:105F100070B5054600F092FE0646184C0AE0681C73
:105F200008D0002D04D000F089FE801BA84201D9C2
:105F3000032070BDA069C007F1D1A069800701D519
:105F40000220A061A069C00511D4A06980050ED40B
:105F5000A06940050BD4A069000508D4A06980049D
:105F600005D4A069800302D4A069C00303D5FFF75C
:105F700087FF012070BD002070BD0000002002409E
:105F8000F8B51746002605460C4600F04BFD09E023
:105F900029460220226800F027FD002804D1241D94
:105FA0002D1D361DBE42F3D300F010FDBE4201D2BE
:105FB0000020F8BD0120F8BD10B5084902460020B8
:105FC000054B497905E044001C5B944203D0401C1A
:105FD000C0B28842F7D310BD6C13002070000020BF
:105FE00010B500F01CFE10BD10B5094801F012F804
:105FF00080B2FFF7A3FB074A074BFFF783FA0022A3
:10600000064BFFF7E7FAFFF7F9FB80B210BD00007F
:10601000E4150020F853E3A59B843E4000408F40E8
:1060200070B53A493A4A00208300401CC0B2D150B2
:106030001428F9D3384937480A78027549784175E8
:1060400036490A780276497841763249052013317B
:1060500048720A2005F0A4FA7D20C00005F0BAFAC3
:106060002C49002213310C2005F084FB00210C2068
:1060700005F092FB022005F0E3FA274D284C203D65
:1060800000210F2005F00CFA20426863F8D0686BFD
:10609000411C38D0400435D58122D20100210F2087
:1060A00005F03DFB0021102005F0FAF941061848E3
:1060B000490E0022C43805F029FA154CC43C607A18
:1060C00005281FD102221549601DFFF77BF8002823
:1060D00018D11148A67C6E710422611C3030FFF784
:1060E0004DF821461331084672000C465130FFF737
:1060F00045F868792146420005484838FFF73EF8E0
:106100000320287070BD04F019FB0000FFFF0100A0
:10611000CC13002041120020900000204C010020F0
:1061200000D0272410B5144C1448224610321146D2
:10613000083904F073FD0022114BE168A068FFF7F5
:1061400049FA104A104B05F047FC00220F4BFFF7AD
:10615000D1F900220E4BFFF7D5F9FFF7A9FB20601C
:1061600000221346E168A068FFF77AFB01D020689F
:1061700010BD0020206010BD00000020880100201C
:1061800000AA8F406C45D9CC955BC83F0000F03F1A
:1061900040A5E54010B5084800F096FA0A210648E7
:1061A00000F032FA044800F01DF9800503D50248DA
:1061B00000F01AF980B210BD88150020F8B52F4DF7
:1061C00000220121284600F032FDFFF7E3FFFFF730
:1061D0009AFA2B4E3146FFF798F82A4C0122A0601C
:1061E0001146284600F023FD2749A0680025884273
:1061F0003EDB2078254F002815D02570FFF7CAFF19
:10620000FFF781FA3146FFF780F8A060FFF714FB33
:1062100000223B46FFF768F900221D4BFFF772F999
:10622000FFF746FB6060A068FFF706FB00223B46D5
:10623000FFF75AF9174A184BFFF764F906460F465D
:106240006068FFF7F9FA134A144B5242FFF75AF904
:1062500032463B46FFF7A4F8FFF72AFB104960607F
:10626000884201DD616004E0FF21C905C84200D316
:1062700065606068FFF789FAC0B2F8BD000400509D
:1062800000401B44480000200000604000000C401B
:1062900000E064403333333333B33040CCCCEC3F95
:1062A0000000C842F8B5054604464035287C002663
:1062B000012808D001202874206881688907890F87
:1062C00001290ED101E00220F8BD0168C90708D0FC
:1062D000606D202108436065012600202874304647
:1062E000F8BD616DFF2201329143022211436165C5
:1062F000C1688907890F0091C16889088900C16058
:106300002068816892071143816000F097FC07467E
:106310000EE000F093FCC01B0A2809D9606D022131
:106320008843102108436065002028740120F8BDCF
:10633000206880680028ECDB2068C168009A11435F
:10634000C160606D80088000401C6065C5E700008A
:10635000F8B506460D464036317C01290DD00121A5
:10636000317401688A68520709D5416D20221143B2
:106370004165002030740120F8BD0220F8BD174BA4
:106380006A68D80547109A42154C8A6A2B6812D061
:106390005B035B0B1A438A622968490305D5A16830
:1063A0000143A1600A20FFF70DFC2868800312D585
:1063B000A06838430EE05B035B0B9A438A6229684E
:1063C000490302D5A1688143A1602868800302D5F2
:1063D000A068B843A06000203074F8BD0110000030
:1063E00000270140406D70470068006C7047000056
:1063F00070B5040006D0606D2646002540360028A2
:1064000002D006E0012070BDA5653574204600F07D
:10641000D3F8606DC00603D421688868400705D5AD
:10642000606D1021084360653574EBE7606DFF22F5
:106430000132904302221043606588688207920F00
:106440005B48012A02D10A68D2072BD10323626874
:106450009B079A4205D05B429A4202D05B009A4267
:1064600009D10A69920092080A6121680A69636881
:106470001A430A610CE00A69920092080A61816875
:106480000F229204914381608168626811438160A8
:106490002168CA6818239A43CA602168CA68A36839
:1064A0001A43CA6081680122520691438160816863
:1064B000A28E52061143816020688168C90004D40D
:1064C000816801221207114381602068C168394A3E
:1064D0001140C1602069E168022825D000200143F5
:1064E000204620300278037B52035B001A4311439D
:1064F000226B1143A26992031143E269D203114353
:106500002268D3681943D160616A0A46FF3AC23AE9
:1065100005D0A26A11432268D3681943D16042783A
:106520000121012A02D00BE00420D8E700780028DE
:1065300023D0606D202210436065A06D0843A065E4
:10654000E06B012820681FD00169C90703D00169E9
:1065500049084900016120684169C908C9004161D1
:1065600020684169A26B11434161A565606D800897
:106570008000401C6065002070BD2068C268012357
:106580001B041A43C260DBE70269FF239B009A43A6
:10659000026120680269236CA66C1A43636C334362
:1065A0001A430261206802690A430261D3E70000CE
:1065B000002701401902FEFF10B586B004461421E1
:1065C0006846FEF7F4FD0E492068884216D10D4852
:1065D000416B421511434163C16A01221143C162FB
:1065E000C06A694610400590022000900320019087
:1065F000002002900520000700F050FA06B010BD00
:106600000024014000100240F8B5044640692546C8
:1066100040350E4608280BD02068C068C00709D056
:10662000606D202108436065002028740120F8BDBA
:10663000082700E00C2700F001FB009011E0701C1F
:106640000FD0002E05D000F0F9FA0099401AB042A0
:1066500007D9606D04210843606500202874032079
:10666000F8BD206800683842E9D0606D0121490218
:10667000084360652068C16809058A0F0C21002A5B
:106680001BD12022125D002A17D10268120714D5EF
:10669000826853070122002B08DB43688B43436069
:1066A000606D130298431043606506E0606D20231F
:1066B00018436065A06D1043A065A069002801D152
:1066C000206801600020F8BD70B5044621680020F4
:1066D0008968490721D425464035297C01291CD0E9
:1066E00001212974E169012904D02046FFF77CFAD1
:1066F000002811D1616D0A4A1140FF220132114375
:1067000061650021A165297422681C21116021683E
:106710008A6804231A438A6070BD022070BD00009D
:10672000FEF1FFFF30B5014620314A790023022AED
:1067300004D00422C2630B71012030BD02681468CA
:106740000E25AC4314600268146864086400146089
:10675000446C1C22144001221546006CA540456083
:106760004A7118460B7130BD70B5002401462031C6
:106770004A79022A03D00421C163012418E0026887
:1067800013680E25AB431360026813685B085B0057
:106790001360436C1C221340012215469D40036C7C
:1067A0005D604A7100220A71816B002900D0884720
:1067B000204670BDF0B4016C0D6801680C68466C31
:1067C0001C2304221E401746B7402F420ED06707F5
:1067D0000CD50C68A40602D40C6894430C60416C80
:1067E00019408A40016C4A60016B1AE00227B740E9
:1067F00002462F402032002F17D0A70715D50C686E
:10680000A40605D40C680A25AC430C600121517123
:10681000446C02211C40036CA1405960002111719D
:10682000C16A002918D0F0BC08470827B7402F429A
:1068300012D0240710D50C680E25AC430C60446CB4
:1068400001211C400B46A340046C6360C16351717D
:1068500000211171416BE4E7F0BC704770B5040092
:106860003CD01F48256814212818FEF741FC800001
:1068700060641C4820640221204620300246417199
:1068800029681948E3680140A068666918432369CC
:1068900033431843A3691843E3691843236A184331
:1068A000084328600121A0688903884210D00D4860
:1068B0008030836A656C1C210D400F26AE40B343C7
:1068C0008362656C63680D40816AAB400B438362F1
:1068D0000020E06301215171107170BD012070BD75
:1068E000F8FFFDBF000002400F80FFFFF8B504462F
:1068F0008C46203001790025012909D00126067136
:1069000041790027012905D0077102252846F8BDE5
:106910000220F8BD02214171E7632068016849083F
:106920004900016061462046FFF7CEF9206B002840
:106930002068016801D00E2205E004229143016025
:10694000206801680A221143016020680168314310
:106950000160DBE7F8B51A4E0546307C0F4601288A
:1069600007D0012030741748FFF7D2FA010002D097
:1069700021E00220F8BD0020C04338606C6814E0BC
:106980002046FFF743FA0F48FFF7C2FA01460E48C8
:10699000426808239A434260426843159A43426022
:1069A000002901D03C6006E08034A8686A68C00114
:1069B0008018A042E4D8002030740846F8BD0000DA
:1069C000C017002050C30000002002400548416865
:1069D00002221143416041680122114341600020BD
:1069E0007047000000200240F8B50C4C1646207C91
:1069F0000F46012808D0012020740948FFF788FAC3
:106A00000025002802D006E00220F8BD65613E6046
:106A10000348FFF77DFA2574F8BD0000C017002079
:106A200050C3000011484168C9070BD0EFF3108133
:106A300072B60F4AC2600F4AC26081F31088416883
:106A4000C9070ED1416889070DD5EFF3108172B6E1
:106A5000094A0261094A026181F31088406880078F
:106A600001D501207047002070470000002002403F
:106A7000EFCDAB8905040302BFAE9D8C1615141330
:106A80007047000010B504494A69024202D04861CB
:106A9000FFF7F6FF10BD000000040140FCB5002325
:106AA0000124A2E027462A469F403A406FD04D6815
:106AB000012D05D0022D03D0112D01D0122D16D19C
:106AC00085680326AC465D00AE46AE406546B543DC
:106AD000AC46CE687546AE4065462E438660466835
:106AE0000D79BE43ED06ED0F9D4035434560C66808
:106AF0005F000325BD40AE46AE4335468E68BE40BE
:106B00002E43C6604E68022E01D0122E14D1DE082C
:106B1000B60036180196366A5D07B446EE0E0F25AC
:106B2000B54000966646AE43B4460D69009EB5403A
:106B300066462E43019D2E6206687546AE430D796A
:106B4000AD07AD0FBD40354305604D68ED004BD539
:106B5000294D6E6B26436E639E08284DB60075194D
:106B6000AC46AD689E07360F0F27B740BD430527DB
:106B70003F07B84201D1002715E0214FB84201D1AB
:106B8000012710E01F4FB84202D102270BE02BE093
:106B90001D4FB84201D1032705E01C4FB84201D177
:106BA000052700E00627B7402F436546AF60184D24
:106BB0002E684F689643FF0300D516432E606E681B
:106BC0004F689643BF0300D516436E60AE684F68AA
:106BD0009643FF0200D51643AE60EE684F689643B9
:106BE000BF0200D51643EE605B1C0A681546DA400A
:106BF00000D057E7FCBD000000100240000001403B
:106C00000004005000080050000C0050001C005010
:106C1000000401400069084000D00120704742692B
:106C200013460B401B0491430B4383617047002ABA
:106C300001D081617047816270470000014880681F
:106C400070470000700100200248816802788918AE
:106C5000816070477001002010B508480024016869
:106C6000402211430160204600F00AF8002801D0BC
:106C7000012401E000F018FA204610BD0020024077
:106C800070B504460D4D7D202978C000FEF730FA1E
:106C900001460B480068FEF72BFA00F09FFE002823
:106CA00009D1042C07D200222146401E00F014FA1C
:106CB00000206C6070BD012070BD000070010020DC
:106CC0007C01002070477047F8B55F4CA078401CED
:106CD000A07001202071E08B401CE0835B4800889D
:106CE00002F05AFE208AFEF70EFD01467F20C00505
:106CF000FEF70BFB564D06462968FEF770FA286032
:106D00000120E16AC005814201DA084603E030460D
:106D1000FEF7BAFAE062FF21C9050025C84200D398
:106D2000E562607800280BD102214A48FFF772FF24
:106D300002004949494818D00022FFF778FFE5636F
:106D400002214448FFF766FF454F464E002855D0C4
:106D5000E563B08AFEF7D7FC3D490968FEF7C4FD3C
:106D60005FD24149012008705DE00122D1033B4818
:106D7000FFF75DFF208AFEF7C6FC01467F20C005B5
:106D8000FEF7C3FAE16BFEF72AFA3849E06388425E
:106D9000D6DD34480127F926403000900A213046DC
:106DA000FEF7A6F9002903D12B492C48FFF718F963
:106DB00002212848FFF72EFF002801D0002701E01C
:106DC000002F12D102212348FFF724FF00280CD105
:106DD00004F0CAFD00990120888005F021FB6420A1
:106DE00003F08CFE23492248C8600A2003F086FE87
:106DF0003046761EF6B20028D0D1A1E7208AFEF7F1
:106E000082FC01467F20C005FEF77FFAE16BFEF7AA
:106E1000E6F91949E06388429BDB16491448C860CB
:106E200097E711480570708F401EFEF761FC084916
:106E30000968FEF759FD05D86079002802D00120C5
:106E40003870F8BD3D70F8BD240100208E00002090
:106E50006C01002000040050008000000000005081
:106E600084000020E00D002076000020000040405B
:106E70000400FA0500ED00E00000A04070477047F4
:106E8000704710B5044600680168C943C90708D1B6
:106E90008168C943C90704D1012141602046FFF739
:106EA00013FF20680168C943890708D48168C94372
:106EB000890704D4022141602046FFF703FF2068C0
:106EC0000168C943490708D48168C943490704D404
:106ED00004214160204600F0E5F820680168C943BC
:106EE000090708D48168C943090704D4082141600F
:106EF0002046FFF7C3FF20680168C943C90608D4CC
:106F00008168C943C90604D4102141602046FFF7B7
:106F1000DAFE20680168C943890608D48168C9433C
:106F2000890604D4202141602046FFF7A9FF20688C
:106F30000168C943490608D48168C943490604D495
:106F4000402141602046FFF79AFF10BDF8B50400CC
:106F500005D025462035A87B002802D006E0012078
:106F6000F8BD00206873204600F03CF80220A873AA
:106F70002068C26884466368012B01D106208243E1
:106F800016486169814202D0072040038243002BEA
:106F900001D1D82082431248A668024018463043E7
:106FA000676A266A3E433043A66A30431043002B8B
:106FB00002D0012B04D005E02369E2691A4300E006
:106FC000E2681043054A914202D0A2691143084386
:106FD0006146C8600120A8730020F8BDFFFF0000D3
:106FE000F8F119FF10B50068084988420CD108482B
:106FF000816BC20411438163002201210D2000F046
:107000006BF80D2000F05CF810BD0000007C004023
:10701000001002400068C06970470000F8B50446DF
:107020000220254620351746A8731D480268C30470
:107030001A4302602068C2689B121A43C26020682B
:1070400002690126324302612268102050602068E4
:1070500081611021204601F005FC03281FD0216822
:1070600008204860206847610821204601F0FAFBAB
:10707000032814D0204601F085FBA87B03280ED0FE
:107080002068816831438160206801693143016172
:1070900020680169042211430161AE730020F8BD2C
:1070A00000040140704700000448416B0122114375
:1070B0004163816B020411438163704700100240F9
:1070C000002805DBC106C90E01208840014908607F
:1070D0007047000000E100E010B503F00DFB10BDAB
:1070E000024801688215114301607047007000403A
:1070F000F8B5044600780027534D800671D5524EEE
:10710000403EB06BC00004D4B06BA9050843B06327
:1071100001274E480168C90511D401688215114341
:107120000160FFF78BFD009005E0FFF787FD0099F8
:10713000401A642837D845480068C005F5D532683C
:107140000321090560680A400140914208D081038B
:10715000890F032904D13168890301D50120F8BDC5
:107160002A69032109040A4022D0084090421FD016
:10717000207880061CD528692A6988430121C90422
:107180000A432A612A698A432A612861C0050FD50A
:10719000FFF754FD009008E0FFF750FD0099411AF9
:1071A0002B48814201D90320F8BD28698005F3D519
:1071B00061688803800F032805D132680005824387
:1071C00001400A43326028690322616812041140B9
:1071D00008432861002F04D0B16B012000078143D0
:1071E000B1632078C00705D0E868A16880088000F6
:1071F0000843E8602078800705D5E8680C218843BB
:10720000E1680843E8602078400706D5E868032174
:107210008902884321690843E8602078000706D581
:10722000E86803210903884361690843E86020781E
:10723000000606D5E868032189048843A16908434C
:10724000E8600020F8BD00004010024000700040DF
:1072500088130000F8B50E46050038D05E48006877
:10726000C007C00FB04214D25B4C206840084000F9
:1072700030432060FFF7E2FC074605E0FFF7DEFC45
:10728000C11B564881427AD82068C007C00FB0425F
:10729000F4D12878524C800705D5E068F021884366
:1072A000A9680843E0602878C00752D068680228BF
:1072B00006D0032807D0216801280AD0890504E0F8
:1072C0002168890301E021688901002903DB01208D
:1072D000F8BD4907F9E7E168890889000143E160E1
:1072E000FFF7ACFC0746686802280AD0032814D0D0
:1072F00001281ED029E0FFF7A1FCC11B37488142BD
:107300003DD8E0680007800F0228F4D121E0FFF7A4
:1073100095FCC11B3148814231D8E0680007800FDD
:107320000328F4D115E0FFF789FCC11B2B488142EB
:1073300025D8E0680007800F0128F4D109E0FFF7A5
:107340007DFCC11B2548814219D8E0680007800FE9
:10735000F5D121480168C907C90FB14217D90168A1
:107360004908490031430160FFF768FC074608E01F
:1073700005E0FFF763FCC11B1848814201D90320D7
:10738000F8BD15480068C007C00FB042F1D1287899
:10739000400706D5E068072109028843E9680843E9
:1073A000E0602878000707D5E0680721C902884314
:1073B0002969C9000843E06000F03AF8E168094A29
:1073C0000906090F515CC840074908600748006872
:1073D000FFF756FCF8BD00000020024088130000B3
:1073E00000100240FAC500087C0100207401002052
:1073F000044805490068C968044A4905490F515CB9
:10740000C84070477C0100200010024013C60008ED
:10741000044805490068C968044A8904490F515C59
:10742000C84070477C0100200010024013C60008CD
:1074300070B51A4AD3681A490C2018408D000428E8
:107440000CD04E00082810D00C2810D05068000432
:10745000410F0120C003491C884070BD1068C00660
:1074600001D5084670BD284670BD304670BD9802F3
:107470000C4C000F205C1B029C0FD368641CDB03C8
:1074800001D5314603E01268D20600D4294603F044
:10749000F8F822460023FDF741FE70BD00100240BF
:1074A00000093D000AC60008FEB505007ED0FE4C6E
:1074B000E7680C20E66807400120000406402878B1
:1074C000C00747D0082F05D00C2F0AD10120000497
:1074D000864206D1206880033CD568680028E5D044
:1074E00038E0012069680004814203D1216801432A
:1074F000216011E0052301221B04920499422168B6
:1075000002D111432160F1E78143216021680140EC
:107510000091206890432060686800280DD0FFF734
:107520008DFB009005E0FFF789FB0099401A642865
:107530007BD820688003F6D50CE0FFF77FFB009036
:1075400005E0FFF77BFB0099401A6428F0D820681B
:107550008003F6D42878800756D50923E868042FDD
:107560000DD00C2F01D1002E09D000283CD021686D
:10757000994301432160FFF761FB064628E021683B
:10758000490701D5002891D061681F22120291435A
:107590002A69120211436160216899430143216005
:1075A000FFF746FFE16809060A0F00E08BE1BF49DB
:1075B000895CC840BE490860BE480068FFF760FBB0
:1075C000002873D120E0FFF739FB801B0228AFD8D9
:1075D00020684007F7D560681F21090288432969A0
:1075E0000902084360600FE0206840084000206006
:1075F000FFF724FB064604E0FFF720FB801B022870
:1076000096D820684007F7D42878C00660D5002FA8
:107610000CD0A86900284AD02068FF210131084316
:107620002060FFF70BFB06462EE0C1E020688005D6
:1076300002D5A8690028A6D06068072149038843BD
:10764000296A084360606068297F0002000A090611
:1076500008436060286A410B0120C003491C884030
:10766000E16809060A0F9149895CC84090490860A1
:1076700090480068FFF704FB002817D128E0FFF7C7
:10768000DDFA801B0228A2D820688005F7D5606843
:10769000072149038843296A084360606068297F9D
:1076A0000002000A09060843606011E0E2E0216878
:1076B000FF20013081432160FFF7C0FA064604E055
:1076C000FFF7BCFA801B022872D820688005F7D427
:1076D0002878794E000724D568690028306910D0D1
:1076E000012108433061FFF7A9FA009005E0FFF798
:1076F000A5FA0099401A02285AD830698007F6D5B1
:107700000FE0400840003061FFF798FA009005E074
:10771000FFF794FA0099401A022849D83069800787
:10772000F6D42878400766D500200290A06BC000F0
:1077300006D4A06B012109070843A0630120029031
:107740005E480168C90511D40168821511430160C2
:10775000FFF774FA009005E0FFF770FA0099401AFD
:10776000642825D855480068C005F5D5FF20AA68CB
:107770000130824203D131690143316111E00121BD
:107780008902002A07D005231B029A4203D13269DD
:107790000A433261EFE732698243326130698843DC
:1077A0003061A868002810D0FFF748FA009008E080
:1077B0005FE0FFF743FA01460098091A404881420A
:1077C00057D830698005F4D50DE0FFF737FA0090FF
:1077D00006E0FFF733FA0099411A3948814248D848
:1077E00030698005F5D40298002804D0A06B0121EF
:1077F00009078843A063686A002866D00C2F3ED032
:10780000012636060228206805D0B0432060FFF725
:1078100015FA05462FE0B0432060FFF70FFA074640
:1078200004E0FFF70BFAC01B022822D82068800171
:10783000F7D4E96AA86AE2680843296BFD231B04B0
:107840009A4311430843E060206830432060FFF70B
:10785000F5F9054604E0FFF7F1F9401B022808D8C6
:1078600020688001F7D530E0FFF7E8F9401B0228D7
:1078700001D90320FEBD20688001F5D425E0012850
:10788000F8D0E06801210904AA6A014091421AD1A6
:107890000F218904EA6A0140914214D1032189052C
:1078A0000840296B88420DE000100240FAC500082C
:1078B0007C01002074010020401002400070004054
:1078C0008813000001D00120FEBD0020FEBDF8B5E8
:1078D00004000ED0FF27606A0537002500280AD073
:1078E0002561656126464036A562707C002807D078
:1078F0000AE00120F8BD6068B842F3D0E561F1E725
:107900003574204600F03EF8022171742068026848
:1079100040239A4302602123A26860689B021A40B8
:1079200038401043E3688A021340184323690B4030
:10793000217D1843C907C90F0843A1699310194055
:107940000843E169382319400843216A802319401C
:107950000843A16A93001940084321680860A069A0
:107960000421000C0840616A102319400843216873
:1079700048602068C1699143C161656501207074E8
:107980000020F8BD10B586B0044614216846FDF706
:107990000EFC10492068884219D10F48416B8214AF
:1079A00011434163C16A01221143C162C06A0021CF
:1079B00010400590E02000900220019003200390E9
:1079C00002910491052069460007FFF767F806B0A9
:1079D00010BD00000030014000100240094910B500
:1079E000401E884201D9012010BD074C606103216F
:1079F000081F02F081FE0020A06107202061002006
:107A000010BD0000FFFFFF0000E000E0F0B50246FF
:107A10002032137E012B1ED00125157602235376CA
:107A200006687468B3687027BC430F6827437760A3
:107A30000068AC07A04205D0084CA04202D0084C18
:107A4000A04204D180244968A3431943816055763C
:107A500000201076F0BD0220F0BD000000080140BB
:107A60000014014070B5050005D02C462034607E1E
:107A7000002802D006E0012070BD002020762846B4
:107A800000F010F802206076291D286802F04CF8FA
:107A90000120A077A076E0762077607760760020DE
:107AA00070BD0000006801218907884204D10348A5
:107AB000816B012211438163704700000010024076
:107AC000F8B5054604462035287E012817D0012642
:107AD0002E7602206876226890687727FF23B843C5
:107AE0001B02984390600A68502A31D00EDC202A8D
:107AF0004BD006DC002A48D0102A3AD145E00220BB
:107B0000F8BD302A41D0402A33D136E0602A27D050
:107B1000702A12D001200003121A2AD0824228D1E2
:107B2000CB684A688968206802F037F82068816865
:107B300001229203114381601BE0CB684A68896887
:107B4000206802F02AF8216888683843886010E0CD
:107B5000CA684968206802F09AF85021206806E057
:107B6000CA684968206802F0A3F86021206802F022
:107B70001FF86E7600202876F8BDCA68496820682C
:107B800002F085F840212068F1E711462068EEE711
:107B900010B586B0044614216846FDF708FB0121A4
:107BA00020688907884212D10A49CA6A0220024322
:107BB000CA62C96A01900140059141020091002109
:107BC00002910391049069460348FEF767FF06B0EF
:107BD00010BD00000010024000040050F8B5064639
:107BE00004462036307E0D4601280BD001200827A0
:107BF0003076002A08D0042A16D0082A2AD00C2A67
:107C00004DD137E00220F8BD206801F0D9FF20688F
:107C100081693943816120688169042291438161CE
:107C200020688169EA6812E0206801F0E1FF2068BD
:107C300081690122D2021143816120688269012198
:107C400089028A43826120688169EA6812021143CD
:107C5000816124E0206801F0E4FF2068C1693943B4
:107C6000C1612068C16904229143C1612068C16972
:107C7000EA6812E0206801F0EFFF2068C169012284
:107C8000D2021143C1612068C269012189028A437D
:107C9000C2612068C169EA6812021143C161002013
:107CA0003076F8BD70B5050005D02C462034607ED6
:107CB000002802D006E0012070BD00202076284672
:107CC00000F00FF802206076291D286801F02CFFD3
:107CD0000120A077A076E07620776077607600209C
:107CE00070BD704770B505462C460220203400292F
:107CF00008D004290BD008290ED0627F012A10D0A9
:107D0000012070BDA27E012AFAD1A0760AE0E27EAF
:107D1000012AF5D1E07605E0227F012AF0D1207713
:107D200000E060770122286801F02AFF012228681C
:107D300092070121904205D0074A904202D0074A9B
:107D4000904204D182685207520F062A02D002687C
:107D50000A430260002070BD000801400014014089
:107D600070B504460D460068002201F009FF206846
:107D7000016A0C4A114203D10168490849000160B7
:107D800001202034002D06D0042D06D0082D06D069
:107D90006077002070BDA076FBE7E076F9E72077FA
:107DA000F7E70000111100007047704770470000AE
:107DB000F8B502680446D06911689668814B05469B
:107DC0001D402023002D6CD0F7077F4DFF0FBC46D0
:107DD0000D402F4379D02546C7078035002F06D0A8
:107DE000CF0504D5012717622A683A432A60820723
:107DF00008D5F20706D0276802223A622A680427CB
:107E00003A432A60420708D5F20706D026680422C2
:107E100032622A68022632432A6002070AD50A46DD
:107E20001A406646324305D02668082232622E6820
:107E300016432E60020508D54A0106D501222668A0
:107E4000D20232622A681A432A602A68002A30D095
:107E5000800606D5880604D5616E002901D020462B
:107E60008847286821688968490602D42821084281
:107E700025D0204602F04BF920688168490619D5C3
:107E8000826840218A438260206F002812D04F49C7
:107E90008163206FFEF768FC00280AD0206F816B99
:107EA00006E0850611D58D060FD5616E77E0204678
:107EB0008847F8BD2046FFF779FFF8BD05E020466A
:107EC000FFF774FF00202860F7E7256E012D56D1DB
:107ED000C50654D5CD0652D5102616622068816895
:107EE00025464906403500292ADA226F116849687B
:107EF0000904090CE1D02F8B8F42DED96983116808
:107F00000968890617D4016832019143016020682D
:107F10008168490849008160206881684022914356
:107F20008160E3670020206620680168B14301603A
:107F3000206FFEF7F7FB288B698B401A81B21AE09D
:107F4000298B6A8B891A6A8B89B2002AB5D00029DD
:107F5000B3D00268FF252135AA43026020688268F9
:107F6000520852008260E367002020666066206845
:107F70000268B24302602046FFF716FF9DE7C50284
:107F800008D5750206D50120000510622046FFF7CE
:107F90000CFF92E7050605D50D0603D5A16E002955
:107FA00085D18AE7400688D5480686D511682046DF
:107FB0004024A143116083670021816600F043F9EA
:107FC0007BE700000F0800002001000435A0000836
:107FD00010B5040003D0A06F002802D007E00120F4
:107FE00010BD002174200155204600F027F8242000
:107FF000A06720680168490849000160204602F036
:10800000D9F80128ECD0606A002802D0204601F09F
:10801000F1FE206841680922D20291434160206844
:1080200081682A22914381602068016801221143FE
:108030000160204601F044FF10BD0000F0B587B09C
:10804000064614216846FDF7B2F82C49306888428C
:1080500051D12B48416B0122920311434163C16A04
:1080600001221143C162C06A00251040059003201F
:10807000400200900220032701A9A1C1042004901E
:10808000052069460007FEF709FD1F4C1D48A56045
:10809000E56081C48027E560A760202025616061DC
:1080A0000002A0611848083CFEF7D8FB002801D068
:1080B000FDF7AAFE3467A662144C12482146143814
:1080C00020600320606010200831A1C16561A561B6
:1080D000E56120462562FEF7C1FB002801D0FDF7CF
:1080E00093FEF466002201211B20A662FEF7F4FF36
:1080F0001B20FEF7E5FF07B0F0BD0000003801408F
:108100000010024030000240301700207817002095
:1081100070B5C36F202B27D100290BD0002A09D0BE
:10812000012483682403A34206D10369002B03D1F1
:10813000CB0701D0012070BD034660331C7D012CAC
:1081400012D001241C7500230366084C0368A34267
:1081500007D05C68240204D51C680125AD062C43B9
:108160001C6002F027F970BD022070BD004800407D
:1081700070477047FFB50446806F83B017460D46C1
:1081800020285ED1002D0AD0002F08D0A168C001A0
:10819000814207D12069002804D1E80702D00120DC
:1081A00007B0F0BD204660300090007D012848D027
:1081B0000098012101750020802108512120A0672D
:1081C000FEF73CFD2646403601903782778201203B
:1081D000A1680003814202D12069002805D02F4602
:1081E000002500990020087511E00027F9E700221A
:1081F0008021204602F024F9002815D1002F15D047
:108200002168387888627F1C708A401E7082708A6C
:10821000019B002806980090E9D1002240212046C9
:1082200002F00EF9002808D00320B9E72888216859
:10823000C005C00D8862AD1CE6E72020A0670020C5
:10824000AEE70220ACE77047034D044C04A002F0F7
:10825000F7F9E560FAE700000400FA0500ED00E038
:10826000486172644661756C745F48616E646C65E8
:10827000722E0D0A0000000000B585B0142168467A
:10828000FCF795FF03480221418300F015FC05B07F
:1082900000BD00002401002070B501240E4DA40390
:1082A000002221462846FEF7C2FC0022042128466F
:1082B000FEF7BDFC0A2002F028FC012221462846D8
:1082C000FEF7B5FC0A2002F020FC002221462846D9
:1082D000FEF7ADFC70BD00000004005070B5012435
:1082E0000E4DA403002221462846FEF7A0FC0122E1
:1082F00004212846FEF79BFC0A2002F006FC01221E
:1083000021462846FEF793FC0A2002F0FEFB0022DD
:1083100021462846FEF78BFC70BD0000000400508B
:10832000F1B500240126154F2546B603002231463B
:108330003846FEF77CFC0A2002F0E7FB01223146BA
:108340003846FEF774FC6006040E04213846FEF73A
:1083500061FC002801D0641CE4B2052002F0D5FBCA
:108360006D1CEDB2082DE1D30098002803D0FFF773
:1083700093FF2046F8BDFFF7B1FFFAE70004005075
:10838000F8B50126154F0546B6030022314638469A
:10839000FEF74DFC0024E80901D0012200E0002294
:1083A00004213846FEF743FC6806050E0A2002F059
:1083B000ACFB012231463846FEF739FC0A2002F0B8
:1083C000A4FB002231463846FEF731FC0A2002F0B9
:1083D0009CFB641CE4B2082CDDD3F8BD0004005003
:1083E00070B50D4C012204212046FEF720FC01222D
:1083F000950329462046FEF71AFC00220421204658
:10840000FEF715FC0A2002F080FB002229462046D8
:10841000FEF70DFC70BD00000004005070B5012493
:108420000E4DA403002221462846FEF700FC002240
:1084300004212846FEF7FBFB0A2002F066FB01221E
:1084400021462846FEF7F3FB012204212846FEF7C9
:10845000EEFB0A2002F059FB70BD00000004005042
:1084600070B5144D0024012204212846FEF7DFFBDD
:10847000062002F04AFB0122960331462846FEF709
:10848000D6FB062002F041FB07E0641CE4B2FA2CA4
:1084900003D9FFF7C3FF012070BD04212846FEF772
:1084A000B9FB0028F1D1002231462846FEF7BFFB78
:1084B000002070BD00040050F8B501F033FD01F05C
:1084C0006DFD63480068C0696148C838FEF7A2FDC9
:1084D000604C80B2A082A18B421A032A01DC814247
:1084E00006D9A08301210520C9020007FDF778FD08
:1084F00059485A4E808F0025002832D0E16A720315
:108500005748914202DB0221017000E005700078BB
:1085100001218902002805D001280ED0022811D09F
:1085200003281ED1608B01282ED0022819D148487B
:1085300008214038FFF714FC13E0A08AFF22F5322F
:108540009042EFD2608B01281CD0022804D008E0B2
:108550003046FEF76CFB04E03D4808214038FFF749
:10856000C1FBFDF72BFE207040213046FEF752FB89
:108570000127FF0300282DD03A480560E079002844
:1085800004D007E00022E3E70122E1E70120E071E7
:1085900001F0B8FF80213046FEF73CFB002806D0F2
:1085A000002208213046FEF742FB012205E00122AD
:1085B00008213046FEF73BFB002205203946000724
:1085C000FEF735FB244C284E4034A08C274F012861
:1085D00003D01CE0E5710022EAE7254869460880DF
:1085E00072B680212348FDF727FC002804D0022220
:1085F00069462048FDF7C4FC62B61FA002F020F8CF
:10860000A58403F00DFF642002F078FAFE60608C10
:10861000012808D110486584058003F001FF64201B
:1086200002F06CFAFE60208C012806D1258403F04C
:10863000F7FE642002F062FAFE600748124A0188E1
:10864000914202D1C088002800D1FE60F8BD000030
:10865000AC16002024010020E00D00200004005092
:10866000820000206C0100200400FA0500ED00E00B
:10867000AAAA0000384A0008BDF8C8EBC9FDBCB67C
:10868000C4A3CABD0D0A0000AA55000008B55721B1
:10869000202000F06AF80321212000F066F8402134
:1086A000222000F062F80821232000F05EF8AA21C1
:1086B000302000F05AF8084801210187322000F0EC
:1086C00054F80221332000F050F8684600F006F814
:1086D0000A2002F01AFA08BDE00D002010B501468C
:1086E0000F2000F021F8002800D0012010BD10B5A7
:1086F0000446FFF775FE3220FFF742FEFFF7B0FE9B
:10870000E0B2FFF73DFEFFF7ABFEFFF769FE332057
:10871000FFF736FEFFF7A4FE0020FFF701FE044638
:10872000FFF77CFE204610BD10B50C46FFF7DFFFBB
:108730002070012010BD70B50D460446FFF750FEB5
:108740003220FFF71DFEFFF78BFEE0B2FFF718FEA9
:10875000FFF786FE2846FFF713FEFFF781FEFFF7BF
:108760005DFE0A2002F0D1F970BD10B5FFF7E3FFFE
:10877000012010BD10B50248FEF783FB10BD0000BC
:10878000E4150020FEB50446002772B6334A01689E
:108790008B1804D13248C7680320800407408868DA
:1087A0000190C868009048698E69002B08D12C4957
:1087B00040398B6ACD042B438B628B6AAB438B624F
:1087C000014631433CD025492368CB4205D1244999
:1087D000CA6803239B049A43CA60254620350028B3
:1087E00010D021680A6901231A430A61216848618F
:1087F0000821204600F036F8032800D1A87321682C
:1088000008204860002E10D0206801690122114321
:108810000161206886611021204600F023F80328BA
:1088200000D1A8732168102048600C482168C1421B
:1088300006D10B48C1680322920491433943C160B9
:108840002068016949084900016121680198886030
:1088500021680098C86062B6FEBD00000084FFBFBA
:108860004010024070B506460B480D4600240949E9
:108870000068FCF73DFC7D21C90048433168401E7B
:1088800000D103240B682A469A4301D00028F6D170
:10889000204670BD204E00007C0100201CB5002148
:1088A00016480091144A01910260C16312054260AA
:1088B000816007228263012202610246C160203288
:1088C0001170FF235170C2334362816211730163DF
:1088D0008161042241634261C161FDF789FD08485D
:1088E00000908013019069460448FDF731FD002196
:1088F0000248FDF7D7FC1CBD00240140881500206C
:108900000200000408B50848016B0122114301630D
:10891000006B01211040009000220A20FEF7DCFBD2
:108920000A20FEF7CDFB08BD00100240F0B587B06D
:1089300014216846FCF73BFC4648C26A04210A43FE
:10894000C262C26A0A400592C16A80263143C1628E
:10895000C16A31400591C16A01242143C162C16AE3
:1089600021400591C16A02252943C162C06A22469D
:1089700028400590052010210007FEF758F9012234
:1089800035493648FEF753F9002235493348FEF79A
:108990004EF991210520002209020007FEF747F950
:1089A000304801900027052069460297009400078F
:1089B000FEF774F82C4800901120019003200390DA
:1089C000029769462548FEF769F810206A46039524
:1089D00091C2052069460007FEF760F8112001905A
:1089E00002976946039700941C48FEF757F81F4802
:1089F00001906946009502941848FEF74FF8402010
:108A000000906946019702951448FEF747F8184808
:108A1000694691C1694611480397FEF73FF89920CE
:108A20000002694691C10520694600070397FEF7D9
:108A300035F869460948019700960294FEF72EF82A
:108A4000002201210520FEF747FB0520FEF738FB39
:108A500007B0F0BD001002400542000000040050C5
:108A60000830000000001110044000000000211038
:108A70000832000010B50F4C0D482060FF20053073
:108A800060600020A060E06020616061E061012121
:108A9000206249026062A161A0620720E062204674
:108AA000FEF715FF2068016840221143016010BDE8
:108AB000003001401416002010B58AB00024049440
:108AC0000594069407940894012118480994009489
:108AD0000194029489070394016009218460416034
:108AE000046113494461C160FEF7BCFF012000032B
:108AF000049004A90D48FEF7E3FF0C48FFF7D2F8F5
:108B0000089408A909480994FEF780FF60200090A6
:108B10000848019002940822694603940348FFF72D
:108B20005DF80248FFF734F80AB010BD6C1600205B
:108B3000930400005702000000B585B01421684678
:108B4000FCF735FB0E480D490160E1214902416007
:108B500000218160C160016181610C22C1614261BB
:108B60000162302141620121090381634900C1632F
:108B7000FFF72EFA01F0C0FC05B000BD003801403F
:108B8000AC16002070470000F0B589B00A2002F052
:108B900007FD7D20C00002F01DFDFF4C0025A570E3
:108BA000FE48A065A07B0C2801D30B20A073FC48D5
:108BB000E570FC4E00783071FB49A07909784000DF
:108BC0000843217D89000843F071206BF070010A91
:108BD0003172401C20636079F449B0744200C81FB0
:108BE000FE38FCF7CBFA6079F0498200400080192A
:108BF00060311330121DFCF7C1FA60790621420082
:108C000048438019EA491730921CFCF7B7FA2C2028
:108C1000205E002803D0E749098A0818A0856079FA
:108C2000DD49E04EC000203182190B7B53764B7B2F
:108C3000937606227272E04A1D301278B272A27FD9
:108C400032733246133A0B78137549785175002206
:108C5000314602F08FFD60790021C0001D3002F026
:108C60009BFD022002F0ECFCF5712574E5720127F2
:108C700067732573D148FEF7CDF9A0840646E570E9
:108C80006079FCF75BFDCE4ACE4BFCF73BFC01F074
:108C9000D1FE0022BB07FCF783FBFCF7AFFD00060B
:108CA000C10C881980B2F903E084884201D3401ACC
:108CB000E084C54820642079401C2071BF48FEF73D
:108CC000A9F96084B9484C380390FBE1BB48FEF732
:108CD000A1F96084BD4E0BE0B848FEF79BF980B265
:108CE0006084E18C884203D3B94A8918884206D34C
:108CF00000210F2002F0D4FB30426063ECD0606BA7
:108D0000411C21D040047DD58122D20100210F20B9
:108D100002F005FD7D20C00002F05CFC002002F0A6
:108D20000EFC0021102002F0BBFB41069F48490EBB
:108D3000264600226438616502F0E8FB9B486438EF
:108D4000417A0729C1D101E001F0F8FC0222A149D2
:108D5000401DFCF737FA0028B7D102F06EFD7166AE
:108D60003446306602F056FDF166B066F0786A4629
:108D7000401CF0708D486B38017A1170407A507049
:108D800010880290318C88427ED18648924E8C3079
:108D9000C08E308083488C30008FA0838748FEF7D8
:108DA00039F9608402F08EFAFF22A16E5204E06E5F
:108DB0000023891858410206080A10434108490057
:108DC0000090080E0902216760677648636E0A30DA
:108DD000226E02F007FD6079E36E81007148A26E99
:108DE0000818163002F0FEFC6E48636F1230226FD6
:108DF00002F0F8FC6B4808214172E07C002816D094
:108E0000022200E051E1694872495F38FCF7DAF963
:108E100000280CD163482774C771606D6349163808
:108E2000C2B24E3908466274EA30FCF7A7F960799D
:108E3000002280005B491C3002F09CFC607900211C
:108E400080001C3002F0A8FC009802F0A2FB012078
:108E500002F0F6FB607202216048FDF7DBFE00289D
:108E60001FD0002150484F4A01708C324A49508E21
:108E700007908887908E0590C887E06B1146EC318B
:108E800020640860C43900E0CAE06064C97C8C4694
:108E90000907090F032900D0A174616D1C2902D0B4
:108EA00016E00121DEE73F493B4A8C31C98FD1856D
:108EB0003F4A039B083A1B881381884207DD00283C
:108EC00005DD002903D0A07D401CA07500E0A5753C
:108ED00060460009E074257101202F49E07240319D
:108EE000079A0A80059A4A802073A08B3C49FF307C
:108EF000C33080B2A08388420BD949424018A08376
:108F000030887D21401C80B2C9003080884200D367
:108F1000358036887D20C000A18B70434018A06446
:108F200008903048302107782F48E773008848437D
:108F3000FCF7E9FB01900A2031464143E08B3022E7
:108F400007905043081AFCF7D3FB0199FCF7DDF9B1
:108F50007F21C905FCF743F9FCF717FC80B22149D2
:108F60007F1E0880B84201D1012020732685182079
:108F7000205EFCF7CFFB06460391608CFCF7DEFB1E
:108F80001A4A1B4BFCF7BEFA02900F460898FCF7F2
:108F9000C1FB3B46029A2DE0700000203F420F00CB
:108FA0002401002054120020680100206C130020CE
:108FB000A8140020200E002034010020E415002019
:108FC000B81E85EB51B8CE3FA086010000D0272403
:108FD000983A00004C010020640100200004005079
:108FE000E70300004201002046010020F853E3A5FA
:108FF0009B843E40FCF778FA3246039BFCF7D0F99D
:10900000FCF7D8FBE064079800F0C6FC607A002803
:1090100061D100210F2002F043FA0006F9D55AE091
:10902000FCF7CAFF614A03211154FF3A60491D3A17
:10903000538E8B87928ECA87626D1C2A06D15B4B3A
:109040004200AC33D318039A12885A8086005748DE
:10905000584A60383018928F02805448E16B30389B
:10906000301841605348E36E8C3830181630A26EC9
:1090700002F0B8FBA16DE06B884207DA4B4960391A
:109080008959012902D1A0650299069147496039A1
:109090008A59824216DD012A14DD2146002811DD9D
:1090A00002980884022020700CE0324600210F2034
:1090B00002F035FB6079E178401C814202D000204B
:1090C00002F03DFA608CE18C884200D2FEE53A4A1B
:1090D00089188842FAD8E07A012801D00220E0728B
:1090E00002F0F0F8354A00210F2002F018FB207939
:1090F000002811D0324909888A008918814200D29B
:109100002570207C002835D028490C310B78487810
:109110008A78022B16D02DE0216CA26D32392046C0
:109120008A420DDAC179264A491CC9B2C171128836
:1091300052008A42E5D20699018402212170E0E7BB
:10914000E571DEE710280CD0C82813D21D4BC91CCE
:109150001818FCF713F803F063F9642001F0CEFC53
:10916000F2E5194D28684000000E03D1C878FCF7DD
:10917000CAFA28600F4D00208C352E46227861797E
:10918000183607E04300EF5AF35A9F4200D00222FC
:10919000401CC0B28842F5D32270084A00218032B8
:1091A0000F2002F0BCFA09B0F0BD0000FC13002053
:1091B00070000020E0120020983A000000D0272420
:1091C00034010020E00D0020500100207047000015
:1091D000F0B58BB0002005900A2002F0E1F97D2067
:1091E000C00002F0F7F9BE4800218170026BBE4C4E
:1091F000521C0263BB4A838D128A2546D21882858F
:1092000041752146133108912030473103903135A3
:1092100020461338B54F02910690B14E0F21B44845
:10922000717100782071B34AB07912784000104310
:10923000327D92001043E071308EE070000A20729F
:10924000A17431461E2284310898FBF797FF402213
:109250002846A949FBF792FF039902980A7BC2743A
:10926000497B017509206072A44831460078A072DC
:10927000B07F2073707D84314000421806991078C9
:1092800008755078487576200022974902F072FAE6
:1092900070790621484300211C3002F07DFA02203B
:1092A00002F0CEF900210F2002F0FAF83842706384
:1092B000F8D0706B411C18D040047DD58122D201BA
:1092C00000210F2002F02BFA0021102002F0E8F814
:1092D00041068548490E0022B43002F017F9824851
:1092E000B430417A022902D0D3E001F027FA0222F9
:1092F0008349401DFBF766FF0028F5D1784802221C
:10930000407D41007648843009187748B530FBF736
:1093100059FF0028E8D102F090FA714E716630666C
:1093200002F078FAF166B0660598002847D101206E
:109330006D49059073488C31C98E01806A488C3024
:10934000008FB0837048FDF765FE7084B08B6F4965
:10935000FF30C33080B2B08388420DD949424018F3
:10936000B0836848694A01880B32491C89B2018080
:10937000914201D30021018062487D210088C9000B
:10938000B28B41438918B16461490A88D1B2F17343
:109390008C4601460A3909B27185002903DA7D231A
:1093A000DB00C91871856146491E8A4201D101213D
:1093B00031733085F08B00E08CE000F0EDFA4A4824
:1093C00069468C30428E0A80808E4880464904224D
:1093D000B531C81FFF38FBF7D1FE4148464A407DF2
:1093E0000099800011503E48FF23816EC06E5B04DF
:1093F0000022C918504100060E0A0643304602F00A
:10940000C8F8710849000A0E0802354900264A6763
:1094100008670846436E026E3348483802F0E2F9A6
:109420002F48C36E826E3048443802F0DBF92C4876
:10943000436F026F2C48403802F0D4F92A490022C9
:1094400052393C2002F096F900213C2002F0A4F9A8
:10945000012002F0F5F82249487208468078401C45
:10946000887001210520C9030007FCF7B9FD1C48DD
:10947000407A002805D100210F2002F011F80006E3
:10948000F9D5802200210F2002F049F914494E70CD
:1094900002E01349012048701148417D491CC9B2BE
:1094A00041750F2900D2B8E60598002810D10C4864
:1094B0001849C28B002A02D00B889A4201D9098828
:1094C000C1831549C08B0988401E48431349088051
:1094D0000BB0F0BD124A00210F2002F020F9D8E7AE
:1094E00070000020200E00205412002000D02724FD
:1094F00024010020680100205814002034010020BD
:109500004C01002064010020E4150020E703000066
:1095100042010020300100202E0100202C010020FB
:1095200000902724F8B531492F48086002F01CFA52
:109530002F4800F0F1F92F4CE0822D48801C00F0FC
:10954000EBF920832A48001D00F0E6F960832B48E0
:1095500029494180014640310979294F0906090E00
:10956000617006D1C7800121C1870A21418700218E
:109570008187244AC18E1170C18F6171818FA17161
:10958000817AE17085880521A5626181C6883046AF
:10959000FBF7AEFDA08101462846FBF7A9FD880038
:1095A000081885B2164825816843FCF7C7F8164AA3
:1095B000164BFCF70FF8FCF721F9E0816582314684
:1095C0003846FBF795FD20820146C820FBF790FD49
:1095D00060840120E083FCF707FDA082E2890C494A
:1095E0000C48FDF71BFDF8BD31A500086800002000
:1095F000004F00082401002026020000E00D00209A
:10960000E803000018000020F853E3A59B843E40C7
:10961000FF7F0000E4150020F0B5994D85B00120D2
:109620002880984FC820984C3880207A401C20729F
:10963000C00706D0E08B411EE183022801D2C8207A
:10964000E083E08B00F0A8F90A2001F0A9FF7D205B
:10965000C00001F0BFFF02218C48FDF7DBFA0028B3
:109660003FD000208A49800009788B4E490008438A
:10967000884909780843B072102070728748C18801
:109680007D20C000FBF734FD707385488349007866
:10969000B07330460B308A780270C97841707F49C8
:1096A000421C20310B7ED370497E11717B49D01C46
:1096B00022310B7E5371497E9171784940310A7C89
:1096C0000271497C417100223146172002F052F8A4
:1096D0000021172002F060F8022001F0B1FF714E66
:1096E00003E00120BEE7FEF7E7FE00210F2001F0B6
:1096F000D7FE30426063F6D0606B411C7ED04004E0
:109700007DD58122D20100210F2002F008F800212E
:10971000102001F0C5FE41065F48490E0022B4301A
:10972000616501F0F3FE5C4EB436707A112866D1A3
:1097300002225D49701DFBF745FD00285FD1F01F37
:10974000027A69460A70407A4870B17A2980C82046
:10975000FBF7CEFC3880307BE0833046534D283811
:10976000C08E288030462838008FA0835048FDF7EF
:1097700051FC80B260840390A08B4E49FF30C3300F
:1097800080B2A08388420CD949424018A08328881F
:109790004849401C80B20B312880884201D3002008
:1097A00028802D887D20C000A18B68434018A064CC
:1097B00002904148067828460A3800B2E673608570
:1097C000002803DA7D21C9004018608538883021DF
:1097D0004843FBF798FF07462A20205EFBF788FFE7
:1097E0003946FBF792FD7F21C905FBF7F8FCFBF733
:1097F000CCFF314980B20880761E01E03EE03BE0BC
:10980000B04201D10120207325851820205EFBF78E
:1098100081FF074601910398FBF790FF274A284BE9
:10982000FBF770FE05460E460298FBF773FF2A46CB
:109830003346FBF759FE3A46019BFBF7B1FDFBF7B8
:10984000B9FFE06468460088208413481249B430A8
:10985000807CC7316071420008460D465130FBF7ED
:109860008DFC6079294642001648FBF787FCE08BA7
:10987000FF2801D00320207005B0F0BD00F05EFF8E
:109880003401002046010020700000200004005038
:10989000290100202A01002054120020E00D0020A0
:1098A0001800002000D027244C0100206401002073
:1098B000E4150020E703000042010020F853E3A56F
:1098C0009B843E408413002070B586B01421684606
:1098D000FBF76DFC01250F4EED03002229463046B3
:1098E000FDF7A5F901200024019002946946009536
:1098F00003943046FDF7D2F80320019002946946A4
:10990000009503943046FDF7C9F8022001F0F6F8FF
:1099100006B070BD0004005000887047704700001A
:10992000F8B5044600206A461080194D55222A7069
:10993000AA226A700322AA70661DEE702A716971EC
:10994000144A49008918AC712246E81DFBF716FC41
:10995000002007E029186A468978128889186A4623
:109960001180401CB042F5DB611DA81CFCF792F988
:1099700001466846018029190078C8716846407818
:10998000087221460931024800F0E2FBF8BD0000F0
:1099900022150020E00D002010B51B4C228A01E0AA
:1099A000891AE183E18B9142FAD2628C8BB25343E4
:1099B0001B182384132902D14A4310182084208CB9
:1099C000302148436421643048431049A06309684A
:1099D000401A4B21090140186063FBF79BFE0C4ABB
:1099E0000C4BFBF7F7FDFBF7E5FE0B4920638842C4
:1099F00002DD4A4280182063002801DA4018206303
:109A000006490968486110BD24010020BC000020FF
:109A1000F853E3A59B843E40FF7F0000E41500203F
:109A2000034A1168382389B2994301431160704792
:109A30000030014010B5FDF707F910BD10B59AB020
:109A400034216846FBF7B3FB14210DA8FBF7AFFBED
:109A50001C2112A8FBF7ABFB1B4801680324E4029E
:109A6000A143C21489180160FDF73AFB1748016948
:109A7000A143016106200090FF20013002900120E7
:109A80000390102004900220099040040B900001E4
:109A900000240C900A946846FDF706FD0F200D90F7
:109AA00003200E900F941094012111940DA8FDF73E
:109AB000D1FB81201290032080041890149412A8E6
:109AC000FDF716FB1AB010BD0070004040100240B8
:109AD00010480168821511430160C1680E4A1140A7
:109AE000C16001680D4A1140016081684908490060
:109AF000816001680122920491430160C168FD22E6
:109B000012049143C1600021016106490448886044
:109B100070470000001002400C40FF88F6FFF6FE80
:109B20000050000800ED00E070B5026801239B07BB
:109B3000114C124D984203D0A04201D0A84203D14B
:109B40007026B2434E683243984203D0A04201D0FF
:109B5000A84204D103231B029A43CB681A438023F3
:109B60009A430B691A4302608A68C262096881627B
:109B70000121416170BD0000000801400014014056
:109B800010B5CB06DB0E0121046A99408C430462B8
:109B9000016A9A401143016210BD30B58468FF2507
:109BA0002D021B021343AC430B432343836030BDA0
:109BB000826870239A430A4307210A4382607047F0
:109BC00030B5026A520852000262026A456883692F
:109BD0007024A3439C080B68A40023430224A243DF
:109BE0008C6845601443836149684163046230BDF9
:109BF00030B5026A10239A430262036A456882699B
:109C000073242402A2430C682402144320229343A9
:109C10008A68456012011A4384614968816302625F
:109C200030BD30B5026AFF2301339A430262026AF3
:109C30004568C3697024A3439C080B68A4002343B0
:109C400001246402A2438C68456024021443C3616A
:109C50004968C163046230BD30B5026A01231B0349
:109C60009A430262036A4568C26973242402A243CC
:109C70000C68240214430122520393438A6845600E
:109C800012031A43C46149680164026230BD30B5F1
:109C9000036A046A6408640004628469F025AC43C2
:109CA000120122430A24A3430B438261036230BDA5
:109CB00030B5036A1024A34303628469036A0F2545
:109CC0002D031203AC432243A024A34309011943EB
:109CD0008261016230BD0000F8B5102605252D0710
:109CE000AE62AF20800000F010FFFCF71BFA364890
:109CF00034490068FBF7CCFAFBF72EFD334CA08506
:109D0000AE6101F0E1FB324F324EE0650EE001F052
:109D1000DBFBE065FEF7D0FBA06B411CA1631428C0
:109D200004D92DA000F08CFC2F48C760E06DB04234
:109D3000EDD10026A66320780127FF03030000F081
:109D4000B8FC05040C192D30320001223946284692
:109D5000FCF76DFFFFF760FC06E00122394628465C
:109D6000FCF765FFFFF734FA002239462846FCF776
:109D70005EFF18E0A07A0122401EA07239462846F4
:109D8000FCF755FFFCF74CF9002239462846FCF752
:109D90004EFFA07A002806D1267004E0FEF7F4FEFC
:109DA00001E0FFF715FA02211048FCF733FF002805
:109DB00005D000200E49087001F06CFAF8BD0120B2
:109DC000F8E700000000C8420000002070000020FA
:109DD0000400FA053001CADE4457204944204552A8
:109DE000524F522E0D0A000000ED00E0000400501A
:109DF0006801002010B5818CC90707D001684A6846
:109E000001235B049A43836A1A434A60818C890761
:109E100007D501684A6801231B049A43C36A1A43A1
:109E20004A60818C490707D501684A6801239B0471
:109E30009A43036B1A434A60818C090707D501686E
:109E40004A680123DB039A43436B1A434A60818CBF
:109E5000C90607D50268916801231B039943836BE8
:109E600019439160818C890607D501688A680123AE
:109E70005B039A43C36B1A438A60818C490612D5EF
:109E800003685A6801210905046C8A4322435A6019
:109E9000026C8A4207D10268516803235B0599432B
:109EA000436C19435160818C090607D501684A68E3
:109EB0000123DB04806C9A4302434A6010BD00001A
:109EC000F8B50446002680300660FCF7B7FE05466C
:109ED00020680068124F000709D501212B46002297
:109EE00049052046009700F0ABFA00280DD1206804
:109EF000006840070BD501212B460022890520462A
:109F0000009700F09DFA002801D00320F8BD202022
:109F1000A067E0672666603426750020F8BD000063
:109F2000FFFFFF01F8B5184CC826E078002829D1BA
:109F30006079002826D101206071144D686B0027DC
:109F400000281ED0686BC821081A15E01048E16887
:109F5000405C616988470F480A21008848430E49E0
:109F60000880E068401CE060E068C82800DBE7602B
:109F7000696BC820401A761EE168814201D0002E2C
:109F8000E4DC6771F8BD00005400002000000240CE
:109F9000180D0020340100204801002070B5224C2B
:109FA000E07800283FD1207900283CD101202071A1
:109FB0001E4EF16900250906002933DA2156625741
:109FC00091420AD1F06940062CD5A079002829D009
:109FD000A5712089401C208124E0A179002903D1AA
:109FE000A0710A2000F091FD00202056CC214843AA
:109FF0000F494218206912181279B262401C0022DF
:10A000002061A256CC235A43895881420ADC25613B
:10A010002078401C207020780E2800D12570A07870
:10A02000401CA070257170BD540000200038014014
:10A03000F001002010B5806A0022014640314A83B9
:10A040004A82FDF7B3FE10BD70B5846AA06FE56F5C
:10A050002168896800260906002906DA212804D12A
:10A0600052200653204600F06BF8206880684006B6
:10A0700006D5222D04D15A200653204600F047F879
:10A080002046803001681022114301602046FDF710
:10A090008DFE70BD10B501460968806A09688906A1
:10A0A0001CD400225A210A5201680A68FF23013396
:10A0B0009A430A6001688A68520852008A600168FF
:10A0C0008A6840239A438A602021C167016E012972
:10A0D00004D101680A6810239A430A60016E0129BD
:10A0E00002D0FEF745F810BD5821095AFDF75CFE75
:10A0F00010BD10B5806A016E012902D0FEF739F853
:10A1000010BD5821095A4908FDF74EFE10BD0168DF
:10A110000A68FF2321339A430A6001688A6852085B
:10A1200052008A60016E012904D101680A68102377
:10A130009A430A602021C167002101664166704789
:10A1400001680A68C0239A430A602021816770472A
:10A1500070B5164CE278002A0CD12279002A09D178
:10A160000122E2700025C82903DC0222A256002A3F
:10A1700001DCE57070BD0123E356CC2253430C4A49
:10A18000D1500123E356CC2673439B180A4601465F
:10A19000181DFAF7F3FF6078401C607060780E2895
:10A1A00000D16570A078401EA070E2E75400002046
:10A1B000F0010020F8B50446016880682369E6696B
:10A1C00018436369002533431843724A0B68724E83
:10A1D000334003430B602168486803231B03984303
:10A1E000E368184348602168A069914201D0236A5E
:10A1F00018438B680B263602B34303438B606749D1
:10A20000236867488B420CD1C0688007800F06D056
:10A21000012839D0022835D0032821D11EE001279A
:10A220001FE060498B420AD1C0680C21084027D04A
:10A23000042829D0082825D00C2811D10EE09342FB
:10A240000ED1C16803208002014019D00120800294
:10A25000091A19D0091A15D0814201D1082700E046
:10A2600010274F49504840398600934232D1002F81
:10A270000CD0022F0DD0042F10D0082F7FD126E054
:10A280000027EEE70227ECE70427EAE7FDF7B0F83E
:10A2900006E00968C90605D4304603E0FDF7C8F8B2
:10A2A000002872D0626851005118814267D81103AA
:10A2B000814264D3010E0602500800233018594130
:10A2C000FAF72CFF03210902411A384A55E0012010
:10A2D000C003E7E70122E369D20393422BD13B009D
:10A2E00000F0E7F90906090C4D114D4D4D274D00C1
:10A2F000FDF77EF809E0FDF78BF806E00968C9066E
:10A3000005D4304603E0FDF793F800283DD061689E
:10A3100040004A088018FAF7EBFE80B20146244A52
:10A32000103991422BD8511C01400007400F0843BF
:10A3300029E01046EBE73B0000F0BBF90906090CE9
:10A340002112212121232100FDF752F80AE0FDF717
:10A350005FF807E00968C90606D4304604E00EE05D
:10A36000FDF766F8002810D061684A081018FAF75F
:10A37000BFFE80B201460E4A1039914203D9012531
:10A3800003E01046F0E72168C86000206066A06620
:10A390002846F8BD00480040F369FFEF003801404F
:10A3A000401002400044004000093D00FFFC0F0047
:10A3B000EFFF0000F8B5044641654030002627460F
:10A3C000028380373E602220E0672546206F60359B
:10A3D00000281CD01749C162216F17480863216FFC
:10A3E00016484863206F8663236F606D9C46134652
:10A3F0002168024660462431FCF778FA002806D02E
:10A40000102038602E752020A0670120F8BD2E7521
:10A4100020680168FF2201321143016020688168D1
:10A4200001221143816020688168402211438160CC
:10A430000020F8BD95A00008F3A0000849A000087E
:10A44000FFB581B005460F46044660350A9E39E0E7
:10A45000701C37D0FCF7F2FB0499401AB04222D8A6
:10A46000002E20D02068016849072BD5C069C04361
:10A47000000527D401202168C00208622068016815
:10A48000FF22A13291430160206881684908490098
:10A4900081602020A067E06780342060002028755C
:10A4A000032005B0F0BD20680168FF22A13291436E
:10A4B0000160206881684908490081602020A06708
:10A4C000E067EBE72068C1693846884305D0002182
:10A4D00003988142BCD00020E3E70121F8E70000A7
:10A4E00010B504491020096808620248FDF760FCB5
:10A4F00010BD0000AC16002001490D208870704787
:10A500005400002010B507480A22018A5143818473
:10A51000FEF7F8F9FEF710FBC82203490348FDF7E0
:10A52000F7FD10BD24010020180D0020AC160020FE
:10A53000F8B53E4C002321783D4A1D46082910D02D
:10A54000072947D0062950D0052952D0042953D0D5
:10A55000032954D0002956D0012958D002295AD0B5
:10A560005BE0A17800264A1F04E0314FBF5DFB1875
:10A570009BB2761C9642F8DB667927799A195118B6
:10A58000E3786278C9188918C9194018C0430006D1
:10A59000000E1AD1012E14D0022E16D125482449BE
:10A5A000C018FAF7EBFD01F03BFF642000F0A6FABB
:10A5B000BFF34F8F21492048C860BFF34F8F00BFC2
:10A5C000FDE759081046FFF7ABF92570E570A57057
:10A5D000A571F8BDA1795054491CC8B2A071A178E9
:10A5E000491F8842F5D1082001E0607007202070E3
:10A5F000F8BDE0700620FAE760710520F7E7A0706B
:10A60000E5700420F3E7552807D10120EFE7AA28D9
:10A6100003D10220EBE7032803D02570E570A57075
:10A62000F8BD032020702071F8BD00001C0100203F
:10A63000BE140020E00D00200400FA0500ED00E04B
:10A6400010B5024A024900F0E5F910BDFDB7000857
:10A65000800100202021020C01D010211046020AA6
:10A6600001D010460839020901D01046091F82089E
:10A6700001D01046891E420801D0881E7047081A72
:10A680007047F8B5040C8BB2264682B25E430D0CBF
:10A690001046370C5843360480190021794116467C
:10A6A0006E43370C36048019794126466E4389196A
:10A6B000F8BD30B47446641E2578641CAB4200D2E9
:10A6C0001D46635D5B00E31830BC18474900CA02B1
:10A6D0000243100000D004204A0D01D00122104393
:10A6E000044A490D914201D102210843012800D1B9
:10A6F00005207047FF0700008307FF22DB0E9A400A
:10A700008907090E9940002808DB830809489B0047
:10A710001B18186890430843186070470007000F23
:10A720000838830804489B001B18D86990430843E5
:10A73000D861704700E400E000ED00E0BFF34F8F08
:10A7400004490348C860BFF34F8F00BFFDE7000016
:10A750000400FA0500ED00E0F8B504464F1EC800FD
:10A760000838211815461E46086849683A460623E7
:10A770009A4310D02A463346FAF7C4FE3A46D2002E
:10A78000083AA3181A687F1E5B68FAF709FE0622CA
:10A790003B469343EED1022F23D0042F11D0062F36
:10A7A0002FD12A463346FAF7ADFEE36AA26AFAF7DA
:10A7B000F7FD2A463346FAF7A5FE636A226AFAF7DE
:10A7C000EFFD2A463346FAF79DFEE369A269FAF7E0
:10A7D000E7FD2A463346FAF795FE63692269FAF7E0
:10A7E000DFFD2A463346FAF78DFEE368A268FAF7E2
:10A7F000D7FD2A463346FAF785FE63682268FAF7E2
:10A80000CFFDF8BD002210B5134610460149FAF7F6
:10A81000E1FE10BD0000F03F10B5FAF7C1FD10BD1C
:10A82000002210B5134610461146FAF7D3FE10BDAC
:10A8300010B50721024A00200907FAF743FF10BDAF
:10A8400001030000034A10B500201107FAF73AFF90
:10A8500010BD000001FDFFFF02E008C8121F08C183
:10A86000002AFAD170477047002001E001C1121F91
:10A87000002AFBD1704700000149086070470000C2
:10A880008401002008B50021684601706B46012252
:10A8900002212C2000F052FF0221684601706B4615
:10A8A00001222C2000F04AFF08BD000038B5044604
:10A8B0006D20694608706B46012207492E2000F082
:10A8C0003DFF0649002C01D0054A00E0054A2E2034
:10A8D00000F01AFF38BD000006080000061800004E
:10A8E000070600000716000038B504466B46022232
:10A8F0000021362000F0EEFDB3212300FFF7D9FE42
:10A900000E0F08153A3A3A3A1C273A3A2F34483A89
:10A9100000216846017040784108490014E069460A
:10A92000087880088000401C04E0694608788008A8
:10A930008000801C08701DE0684602780A4048329A
:10A9400002704178802001436846417012E06846F9
:10A9500002780A40027040784106490EF4E76946E1
:10A9600048780221084303E069464878FD21084001
:10A97000694648706B4601220021362000F0DEFE59
:10A98000012200AB11463620013300F0D7FE38BD5E
:10A9900069460878CF21084069462030CAE708B5E3
:10A9A000032168464170012101706B46022200219B
:10A9B000362000F0C3FE0122D20306212D2000F034
:10A9C000A3FE012000F09AF80120FFF78DFF08BDDB
:10A9D00008B5020A69464A7008706B4602220421D3
:10A9E0002D2000F0ABFE0320694608706B46012263
:10A9F00006212D2000F0A2FE0020694608706B465B
:10AA0000012206212D2000F099FE0A212D2000F0C0
:10AA100047FD08BDF8B516460F460446002503E07D
:10AA20003946B047641C6D1C20780028F8D12846B0
:10AA3000F8BD0000F8B54A002B4B520DD6182B4A32
:10AA40000C460546142E2BDA002E12DA284BFAF7A4
:10AA5000A7FC00221346FAF717FF40D2002C03DAB6
:10AA60000124E40700253AE02046284337D0214C52
:10AA700014E0214F0B46F7403B402B4331D01C4B99
:10AA8000FAF78EFC00221346FAF7FEFE27D2002CBE
:10AA900003DD01200005F0400419BC4300251EE041
:10AAA000332E1EDC33460027143BFF43DF40384281
:10AAB00017D00F4BFAF71EFD00221346FAF7E4FEFB
:10AAC0000DD2002C0ADD142E0CD03420811B012065
:10AAD00088404019A84200D2641C0546BD43214667
:10AAE0002846F8BD641CF9E701FCFFFF9C7500884F
:10AAF0003CE4377E0000F03FFFFF0F007D2110B5E2
:10AB0000C900484300F001F810BD002140E000BF3B
:10AB100000BF00BF00BF00BF00BF00BF00BF00BF3D
:10AB200000BF00BF00BF00BF00BF00BF00BF00BF2D
:10AB300000BF00BF00BF00BF00BF00BF00BF00BF1D
:10AB400000BF00BF00BF00BF00BF00BF00BF00BF0D
:10AB500000BF00BF00BF00BF00BF00BF00BF00BFFD
:10AB600000BF00BF00BF00BF00BF00BF00BF00BFED
:10AB700000BF00BF00BF00BF00BF00BF00BF00BFDD
:10AB800000BF00BF00BF00BF00BF00BF00BF491C27
:10AB90008142BCD37047FFB581B01E460F4604000A
:10ABA00026D00B9903980143A06A39438268072095
:10ABB0009047002818DB0A99A06A31438268062072
:10ABC0009047002810DB25462035A979032F01D9AD
:10ABD00008200143032E01D904200143A06A8268A2
:10ABE00009209047002806DA0120C04305B0F0BDD7
:10ABF0000020C043FAE7384600F000F920603046F4
:10AC000000F0FCF860600A9868700398A870EF7014
:10AC10002E710B9868710020E8E70000F7B5044634
:10AC2000002090B000900190002C05D06A460621CB
:10AC300001F030FC062803DA0020C04313B0F0BD59
:10AC400068464078010268460078000409186846A2
:10AC500080780818FAF772FD054668460391007976
:10AC600001026846C078000409186846407908184F
:10AC7000FAF764FD032206460F4692075C4BFAF78B
:10AC800003FE07D200225B4B30463946FAF72CFC14
:10AC900006460F4603229207554B28460399FAF7BA
:10ACA000F3FD07D20022534B28460399FAF71CFC08
:10ACB000054603912068FAF741FD02460B463046EF
:10ACC0003946FAF787FC07460A200791205EFAF713
:10ACD00021FD3A46079BFAF715FC06460820099124
:10ACE000205EFAF705FD0021C943FAF74CFBFAF79D
:10ACF000A3FD3246099BFAF753FB06910890606862
:10AD0000FAF71CFD02460B4628460399FAF762FC47
:10AD100005461A200E46205EFAF7FCFC2A4633460A
:10AD2000FAF7F0FB0C9009911620205EFAF7F2FC7E
:10AD3000099B0C9AFAF734FB05910A902A46334690
:10AD400038460799FAF7DEFB059B0A9AFAF7DAFB11
:10AD500005910A901420205EFAF7DCFC3A46079B26
:10AD6000FAF7D0FB07461C200791205EFAF7D2FCC9
:10AD70002A463346FAF7C6FB0E900B911820205E48
:10AD8000FAF7C8FC0B9B0E9AFAF70AFB2A463346E1
:10AD9000FAF7B8FB0B910E902069FAF7BBFC0B9BFE
:10ADA0000E9AFAF7FDFA2A463346FAF7ABFB054648
:10ADB0000E46E068FAF7AEFC2A463346FAF7F0FA98
:10ADC0003A46079BFAF7ECFA059B0A9AFAF7E8FA73
:10ADD00001229207084BFAF795FB02460B46129C9C
:10ADE0000898069903C411980CC0002026E70000BB
:10ADF000FFFF5F4100007041E17A843F00B501210F
:10AE0000C9040300FFF755FC081A05080B0E1114BE
:10AE1000171A0320C00400BD0720C00400BD0F2086
:10AE2000C00400BD1F20400300BD3F20400300BD03
:10AE30007F20400300BDFF20400300BD084600BD49
:10AE4000FEB5264F0D4604000FD0002D0DD026462E
:10AE500000202036B071F07129680D208847002845
:10AE600001DA7800FEBD102801D03846FEBDA5628B
:10AE7000E968002901D028208847204600F030F8F2
:10AE80000028F3DBA06AA52182680E209047A06A03
:10AE9000962182680F209047A06A02218268622072
:10AEA0009047A06A002182680E209047A06A002186
:10AEB00082680F209047717930200191009006231D
:10AEC000202201212046FFF766FE0028CEDB204627
:10AED00000F0AEF80028C9DB0020FEBDFFFFFFFF39
:10AEE00010B586B0044614216846FAF760F9002CC4
:10AEF0007ED0A06A122143686A4610209847122823
:10AF000077D1684600780122010168464078120333
:10AF10000009081843492081884201DD801A2081F8
:10AF20006846837840780007000D181860818842D1
:10AF300001DD801A608168460079012201016846BE
:10AF4000C0781205000309186846407900090818FE
:10AF50003549E060884201DD801AE060684640794A
:10AF60000007030B6846807900021B186846C07909
:10AF700018182061884201DD801A20616846417AF4
:10AF8000007A0002081802B2284801210904A282AE
:10AF9000824201DD521AA2826A46D37A927A120262
:10AFA0009A1812B2E282824201DD521AE2826A46A5
:10AFB000537B127B12029A1812B22283824201DD65
:10AFC000521A22836A46D37B927B12029A1812B2DB
:10AFD0006283824201DD521A62836A46537C127C8C
:10AFE00012029A1812B2A283824204DD501A01E0C2
:10AFF0000BE008E0A083A06A0168282088470028A9
:10B0000006DA0120C04306B010BD0020C043FAE7B5
:10B01000C011C0072034002800D0802060710020BB
:10B02000F1E70000FF070000FFFF0700FF7F0000BF
:10B0300010B5040009D0A06A072182680820904753
:10B04000002805DA0120C04310BD0020C04310BD18
:10B05000072020342070002010BD0000FEB50446FB
:10B060000020019000906079734940000E5A617889
:10B070002578491E7148CFB20163042D77D0072D82
:10B0800075D000210291217801736C49E379012286
:10B0900092058969002B6CD0914381616748217AC0
:10B0A0004173217A82698907890B0A4382610021F1
:10B0B000042000F034FB324661492E2000F024FBCE
:10B0C0003846FFF7F3FB5F4E0522705D81004018A4
:10B0D0005D49431807212B2000F030FB5B490298A3
:10B0E00001220B180B21282000F028FB705D584925
:10B0F00080000A580C21282000F011FBE079554906
:10B1000080004018A1794900425A0221272000F00E
:10B11000FBFA51487E00825B0421272000F0F4FAFC
:10B12000E079002829D0A07804282CD0282069466E
:10B13000087220220621272000F0E6FA02AB012245
:10B140002621272000F0FAFA444938014018E17816
:10B15000890042580821272000F0E1FAA17A601CFA
:10B16000627A0902114313D016E000E001E00121E8
:10B1700088E71143F608816190E7642206212720C1
:10B1800000F0C2FAE0E71020694608720246D1E7F3
:10B1900033490172090A4172417A007A0A02024374
:10B1A0002021272000F0B0FA2E4F0C2123203A68EE
:10B1B00000F0B5FAF01982880421232000F0A4FAE7
:10B1C000A07900280BD0E0792749012243180021FB
:10B1D000212000F0B3FA03200190012000902A07FB
:10B1E000120F10010243607800218007000B024318
:10B1F0000198000502430098400402432079C006EC
:10B20000400902436079C00602431F2000F087FA1C
:10B21000A07861780123084302040848DB03026137
:10B22000E179490319430A4302610021082000F033
:10B2300076FA0020FEBD0000C8C50008B401002059
:10B240000428000070C500082400002042000020EF
:10B2500078C5000898C50008A4C50008A8C500085E
:10B260004110000090C500084400002038B50C468D
:10B2700007498A8B002102432C2000F045FA6846DA
:10B2800004706B46012206212C2000F057FA38BDCD
:10B29000B401002010B5FFF7F5FA10BD10B5044653
:10B2A0000421362000F0FCF80121C902002C01D055
:10B2B000084300E0884302460421362000F02FFABC
:10B2C00010BD000038B540206946087000210E20EE
:10B2D00000F0E6F80446002211460E2000F01FFAA6
:10B2E0006B46012200210D2000F028FA074A0021B8
:10B2F0000F2000F014FA00F0EDF9224600210E2094
:10B3000000F00DFA02480021017338BDF8FF272430
:10B31000D4010020FEB50546042069460870514C52
:10B320000020607521462031206348710873A08396
:10B330006063A06300F0C8F84B4E206002E000F0AC
:10B34000C3F82060B042FAD10020FFF7CDFA00F038
:10B35000BBF8464E20603078242801D9243806E016
:10B360000621F9F7C5FE0622101A4001084302061D
:10B3700001040A4301020A430243B26070600021E3
:10B380001E2000F0CCF900F09FF820606B460122EF
:10B390000021242000F0D2F91E20FFF719FB86B20D
:10B3A000300AA0730420FFF713FB074600F08CF867
:10B3B00020603806000E0DD002206946087101ABEE
:10B3C000012212212D2000F0B9F9A08B01210903DF
:10B3D0000843A08300F078F820600620FFF7F8FA11
:10B3E00060600720FFF7F4FAA060F006C00E207539
:10B3F00001D110202075C0B200F0DCF9E80707D0B9
:10B40000FFF7CDFAA08B0121C9020843A0830AE00F
:10B410000521362000F02EF8154908400246052186
:10B42000362000F071F90120FFF75EFA00210420B8
:10B4300000F036F8A0610021262000F031F8152137
:10B440008903084302460021262000F068F9002203
:10B450002621362000F058F900F036F82060002050
:10B46000FEBD0000B40100203001CADE180000203B
:10B47000FFFD000038B5094C89B280B26B4602224C
:10B4800000F028F8002806D1684640780102684696
:10B490000078081884B2204638BD0000FFFF000085
:10B4A00038B50024E44389B280B26B46042200F030
:10B4B00011F8002806D103216846435C2202D41803
:10B4C000491EFAD5204638BD10B500210846FFF7C1
:10B4D000E7FF10BD38B5002909D0402420436C4651
:10B4E0002070C8B27F2906D8607002200AE0694641
:10B4F0000870012006E0802420436C466070C80973
:10B50000A0700320694600F065FF38BD10B51446F1
:10B5100003460A4621461120FFF7DCFF10BD10B597
:10B520000346052200211520FFF7D4FF10BD10B5FA
:10B530000346052200211720FFF7CCFF10BD38B5C8
:10B54000054600206946087000F0C4F8FF24013465
:10B550002246002D01D00322120200210D2000F00E
:10B56000D3F8002D13D06B46012203210F20FFF7E3
:10B57000B1FF68460078000709D5FFF7A3FE224611
:10B5800000210D2000F0C0F80020C04338BD00208D
:10B5900038BD10B5024601210A2000F0C0F810BDE8
:10B5A00010B5044600211A20FFF77AFF000D220390
:10B5B0000005120B024300211A2000F0B0F810BD64
:10B5C00010B5024602492E2000F09EF810BD000082
:10B5D00004180000F8B505466B460122032104203B
:10B5E000FFF778FF0126114C3607002D0DD02A46B3
:10B5F00000210C2000F088F86946087810210843E3
:10B6000069460870A069304307E069460878EF2171
:10B61000084069460870A069B0430B46A06101224A
:10B620000321042000F08AF8F8BD0000B4010020D6
:10B6300010B502460021182000F066F810BD000089
:10B64000F8B50746002568460570B807204C2E4619
:10B6500000280ADA8020694608706B460122002122
:10B660000D2000F06BF801202073F8076946087878
:10B6700021D006210843694608706B46012200214B
:10B680000D2000F05BF803210F20FFF7F3FE81216E
:10B69000C900084219D04020694608706B46012253
:10B6A00000210D2000F04AF80020FFF7F7FD0025EB
:10B6B0002673ED4309E002210843694608706B4692
:10B6C000012200210D2000F039F82846F8BD0000C5
:10B6D000D40100201CB56B46012203210F20FFF787
:10B6E000F9FE684600784022C1091040C9014000B7
:10B6F000814208D0012069460871024601AB03214E
:10B700000D2000F01BF81CBD08B56B461A70120A1C
:10B710005A7089B280B2022200F010F808BD38B524
:10B7200000236C46E254120A5B1C042BFADB89B23C
:10B7300080B22346042200F001F838BD38B58024D9
:10B74000002909D0C02528436D462870C8B27F293A
:10B7500007D86870022009E020436946087001207C
:10B7600004E020436870C809A8700320694600F00F
:10B77000DBFE38BD10B51446012312189B029A4215
:10B7800002D90020C04310BD0B46821E214609206D
:10B79000FFF7D4FF002010BD10B5054A89051269D6
:10B7A00001430A4300210820FFF7B9FF002010BD24
:10B7B000B401002038B504466B4601220E212B202F
:10B7C000FFF788FE68460078E10640094001C90E8F
:10B7D0000143684601706B4601220E212B20FFF7C2
:10B7E000ADFF38BD10B5002142541C06120A224399
:10B7F0001B0A491C0429F7DB10BD000013B5012307
:10B800001A4669460248FCF7B5FC00981CBD0000CA
:10B81000AC1600207CB5002425466846FFF77FFE65
:10B8200004206946220E2D02154322020C5C1443AB
:10B83000401EF7D5204629467CBD7CB50024254610
:10B840006846FFF774FE04206946220E2D02154358
:10B8500022020C5C1443401EF7D5204629467CBDCD
:10B86000FBF7FAF9FEF7EAF8FDF760F838493948CE
:10B87000002522C005608561C56137490562C16048
:10B880000838FBF763FBFDF73DF8FDF755F9FDF7C9
:10B89000F1F8FDF703F8052601223607D1033046FB
:10B8A000FBF7C5F9FDF73EFEFCF7F0FEFAF7CEF91F
:10B8B000FAF750FAFAF71EFAFCF7DEFC0721B0158A
:10B8C000FFF7D4FCFFF7E6FC244C0A21208A012272
:10B8D0004843A084170339463046FBF7A8F91D48B2
:10B8E000C8221F49C830FCF713FC79103046FAF71C
:10B8F00077FB1C4E2079002827D06078002824D0C0
:10B90000FEF79CF8257120780F2809D901223946C5
:10B910003046FBF78CF9FEF7DFF90022394609E0E3
:10B92000012251033046FBF782F9FEF7D5F90022D8
:10B93000012149033046FBF77AF9FCF7BDFDA08CE5
:10B940000028D7D0401EA084D4E7FCF7B5FDD1E78E
:10B95000007C0040E4150020FFFF000024010020CF
:10B96000180D00200004005010B501229202174962
:10B970001748FAF77BFA1548164902888A4223D0FD
:10B98000018004218180FF21F531C1800A210181DC
:10B9900000211E224181D24382810122C281818302
:10B9A0004323C38602230387782343878287C28782
:10B9B00002464032118451849184C18391801423C2
:10B9C0008382118200F02CFD10BD0000E00D0020EC
:10B9D00000FC0008AA550000F0B51FB496B08446DC
:10B9E0000C460246199D18980390490068006300B0
:10B9F000490840080193002A01D0012600E00026F2
:10BA00009E19FE4BF6185B109E422BD36E00039FCF
:10BA10000296002F00D00127F719F84EF84BBE19F7
:10BA20009E421FD3039E0346F64F334309D03B4645
:10BA30009C4201D1002A04D0019B002A05D0012696
:10BA400004E0002039461BB0F0BD00269E19EE4BE5
:10BA50009E4207D8039F029E002F00D00127F619AF
:10BA60009E4207D92B4660462146189AFEF7D4FE1F
:10BA70001BB0F0BD0023002C29DAE44EB04226DAD8
:10BA8000E34EB04201DB022321E0DE4EB0421EDB7A
:10BA9000E04E070DBE19142E09DD3427BF1B039E8F
:10BAA000FE400196BE40039FBE420BD00FE0039FB5
:10BAB000002F0CD11427BF1B0646FE400196BE4046
:10BAC000864204D1019BDE07F60F02239B1B0E4624
:10BAD000164318D1002D16DA002C03D0022B01D00A
:10BAE000012B06D00220FEF7C7FEFEF78BFE1BB02F
:10BAF000F0BD0220FEF7C0FEFEF784FE0122D20751
:10BB000051401BB0F0BD039E002E61D1BF4EB0422C
:10BB100020D1C148844201D1002A08D0B9488142CD
:10BB200009DB002D10DB189829461BB0F0BD002062
:10BB3000B4491BB0F0BD002D06DA01222946D20718
:10BB4000189851401BB0F0BDB44979440868496861
:10BB50001BB0F0BDAB4FB84225D1002D1FDA002934
:10BB600004D0B14212D1002A09D018E0002A72D1C3
:10BB7000A649E20F0020D20711431BB0F0BD002000
:10BB8000E20F0146D20711431BB0F0BDB14206DA05
:10BB9000234600203946F9F71DFD1BB0F0BD1046C5
:10BBA00021461BB0F0BDB14212DA0126B607B542FC
:10BBB00003D1234610461946FEE3994EB54207D1FC
:10BBC000261E05DB1046314600F040FC1BB0F0BDE0
:10BBD00067007F081646002A40D100290AD08B4A08
:10BBE000914229D1002C0EDD002D1CDB00201146D6
:10BBF0001BB0F0BD022B16D0002C14D0012B12D19B
:10BC0000002C14DB0FE0002C28DA002D09DB012BBF
:10BC100003D000207D491BB0F0BD002081491BB03E
:10BC2000F0BD012B03D0002001461BB0F0BD002069
:10BC30000121C9071BB0F0BD724A91420ED1002C00
:10BC400001DA002B17D0022B06D00020C043F9F7F1
:10BC500061FD1BB0F0BD90E20120F8E7E217521C35
:10BC600094461A4307D000220892664C62465B1E37
:10BC70001A4307D009E00120FEF7FEFDFEF7D0FDD4
:10BC80001BB0F0BD0022644C0892674A90427DDDF3
:10BC9000664B674A98421FDD914202DC002D05DBAE
:10BCA0004DE05848814217DB002D48DD0220FEF7A9
:10BCB000E3FDFEF7BDFD05460E460022534B21462F
:10BCC0000898F9F71FFC084671004908C00FC00723
:10BCD000014328461BB0F0BD914215DA002D2EDA43
:10BCE0000220FEF7C9FDFEF7A3FD05460E46002221
:10BCF000464B21460898F9F705FC72005208C80F18
:10BD0000C0070243114617E03E4B994223DD002D48
:10BD100015DD0220FEF7B0FDFEF78AFD05460E4652
:10BD200000223A4B21460898F9F7ECFB08467100CF
:10BD30004908C00FC007014328461BB0F0BD0220D0
:10BD4000FEF79AFDFEF77EFD49004908E20FD20793
:10BD500011431BB0F0BD002230463946F9F7C4FB51
:10BD6000012205460E46D243F9F7ACFC314A324B6C
:10BD7000F9F7C0FB2A463346F9F7C4FB0022284BEB
:10BD8000F9F7B8FB07462A46334600E064E0039122
:10BD900010461946F9F7B6FB3A46039BF9F7B2FB92
:10BDA0000746032209915207244B28463146F9F7EA
:10BDB000A9FB07910C90224A204B38460999F9F7C4
:10BDC000A1FB074601911F4A1F4B28463146F9F750
:10BDD00099FB3A46019BF9F787FB07460B4602465B
:10BDE000099107990C98F9F7DBFA00250E462846C9
:10BDF000079B0C9AF9F778FB3A4627E0FFFF1F00F4
:10BE0000FFFF0F000000F03F0000E0FF0000F07FA8
:10BE10000000404301FCFFFF0000F0BF5A0B000090
:10BE20000000E03F0000F0FF0000E0410000F043B0
:10BE3000FFFFEF3F555555555555D53F4715F73F32
:10BE4000FE822B6544DF5DF80BAE543E099BF9F78B
:10BE500051FB02460B4652E1012500202D05A94267
:10BE600007DA352230463946F9F72CFC06463420ED
:10BE7000C0430A151218FE48101803900803FD4924
:10BE8000000B01430F46FC49884201DC002003E01F
:10BE9000FA49884202DA0120119005E00020119051
:10BEA0000398401C7F1B039011980597C200F4482B
:10BEB0000F927844801843680268394630460D93E3
:10BEC0000292F9F711FB07910C9030460D9B029AF4
:10BED0000599F9F765FA02460B460020E549F9F79E
:10BEE00079FB09910490079B0C9AF9F70BFB1290D0
:10BEF00000201090E3480D46784400680E90012120
:10BF000078104907084311990D9B890440180121B5
:10BF1000C90447183946029A0E98F9F7E5FA3246ED
:10BF2000059BF9F7E7FA02460B4629461098F9F700
:10BF3000E9FA064602913B4629460E9A1098F9F70F
:10BF4000E1FA079B0C9AF9F7D5FA3246029BF9F70A
:10BF5000CBFA099B049AF9F7D5FA0591129A0A903F
:10BF60002B4610461946F9F7CDFA06460246C64852
:10BF70000F460B4606217844FEF7EEFB32463B4661
:10BF80000091049010461946F9F7BCFA009B049AF8
:10BF9000F9F7B8FA06460F462B461946129A10983A
:10BFA000F9F7FEF9059B0A9AF9F7ACFA32463B46D7
:10BFB000F9F7F6F9109A079104902B4610461946A6
:10BFC000F9F7A0FAB14E0022334609910290F9F731
:10BFD000E7F9079B049AF9F7E3F9002007460246C0
:10BFE00033460091F9F780FA099B029AF9F77CFA37
:10BFF000079B049AF9F77EFA06460D913A462946C0
:10C00000009B1098F9F77EFA07910C902B4630466A
:10C01000129A0D99F9F776FA05460E463A46009BB4
:10C0200005990A98F9F76EFA33462A46F9F7B8F9EE
:10C0300002460B460746099107990C98F9F7B0F9A3
:10C0400000250E462846079B0C9AF9F74DFA3A460A
:10C05000099BF9F74FFA07460722099152078C4BC3
:10C0600031462846F9F74EFA07910090894A884BE5
:10C0700038460999F9F746FA07460191864A874BEF
:10C0800031462846F9F73EFA3A46019BF9F788F916
:10C09000834B7B440F9A9B181A685B68F9F780F909
:10C0A000029009910398F9F735FB05910490099BDB
:10C0B000029A07990098F9F773F97A4B7B440F9A23
:10C0C0009B181A685B6817460393F9F769F9059B93
:10C0D000049AF9F765F90E462846059B049AF9F784
:10C0E00003FA3A46039BF9F7FFF9079B009AF9F721
:10C0F000FBF9099B029AF9F7FDF902460B461999DB
:10C1000000200C900F461898F9F7FCF90291049062
:10C110003B460C9A19991898F9F7E6F92A463346DE
:10C12000F9F7F0F9029B049AF9F73AF909910E90A0
:10C130002A46334639460C98F9F7E4F906460F4685
:10C14000099B0E9AF9F72CF9574A0D46914220DBCC
:10C150005242AA18024310D132463B46F9F7C4F9BD
:10C1600004900391514A524B09990E98F9F718F926
:10C17000039B049AF9F788FB1ED20220FEF77CFB92
:10C18000FEF756FB49004908E20FD20711431BB0E6
:10C19000F0BD6A00474B52089A420DD3464AAA188E
:10C1A000024300D0CBE532463B46F9F79DF9099BA7
:10C1B0000E9AF9F769FBF5D96800002340082C496D
:10C1C0000393020D3D4B5218984223DD01200005D8
:10C1D000521CD04042195000400D40183849794453
:10C1E000096813468C463749C1408B43120301212D
:10C1F000120B090551181422101AC1400391002D89
:10C2000001DA48420390624630463946F9F76CF944
:10C2100006460F4632463B4609990E98F9F7C0F894
:10C2200000252A46284B28460591F9F76BF9079116
:10C230000C90264A264B28460599F9F763F9009198
:10C24000029032463B4628460599F9F74DF9099B7D
:10C250000E9AF9F74FF91F4A1F4BF9F753F9009B54
:10C26000029AF9F79DF807460B460246099135E018
:10C2700001FCFFFF0000F03F8E9803007AB60B0030
:10C280006A070000AC070000D60600000000084066
:10C2900009C7EE3FFD033ADCF5015B14E02F3EBE1B
:10C2A000AA0500007005000000009040FE822B658A
:10C2B0004715973C00CC904000346F3F0000E03FB2
:10C2C000C6040000FFFF0F00432EE63F396CA80CA8
:10C2D000615C20BEEF39FAFE422EE63F07990C98CA
:10C2E000F9F75EF805460E46079B0C9AF9F7FCF83D
:10C2F0003A46099BF9F7FEF809912A4633460E9013
:10C3000010461946F9F7FEF8074602462F480B4635
:10C31000059105217844FEF71FFA3A46059BF9F787
:10C32000F1F82A463346F9F7E5F807460191284621
:10C330003146099B0E9AF9F7E5F8099B0E9AF9F731
:10C340002FF8012304910C9000229B073846019995
:10C35000F9F7CAF805910E903A4628463146019BF6
:10C36000F9F7D0F8059B0E9AF9F734F9049B0C9A6B
:10C37000F9F7BAF82A463346F9F7B6F80022144B13
:10C38000F9F7B8F8064603980D4600054119091556
:10C39000002912DC30462946039AF9F793F9FEF793
:10C3A00095F9042801D1FEF74DFA30462946039A43
:10C3B000F9F788F9064601E004E029180B463246F1
:10C3C00021460898F9F79EF81BB0F0BD68030000FD
:10C3D0000000F03FF0B58C46002510260521090726
:10C3E0008E620E4C08E067467F5DE760A768FF0736
:10C3F000FCD0E7681F706D1C8542F4DB0020074607
:10C4000006E0E760A568ED07FCD0E5681D54401C18
:10C410009042F6D38E610020F0BD00000030014054
:10C4200070B572B60124074DA40221462846F9F7DB
:10C4300003FD002804D0224603492846F9F7A0FD51
:10C4400062B670BD00FC0008E00D0020F8B506469D
:10C450000C46F9F727FB051E0F4600D001200143CB
:10C4600049000B484908411AC90F0DD0002E01D0D0
:10C47000012100E000210C4361004908401AC00F6F
:10C4800002D10120FEF7F8F928463946F8BD000030
:10C490000000F07FF8B515460E460746002407E079
:10C4A0003819C0B200F008F8641C2870E4B26D1CA2
:10C4B000B442F5D33046F8BD10B50446FBF790FF03
:10C4C000EE20FBF75DFFFBF7CBFF2046FBF758FFA5
:10C4D000FBF7C6FFFBF784FFEF20FBF751FFFBF7ED
:10C4E000BFFF0020FBF71CFF0446FBF797FF204629
:10C4F00010BD704770B50D460446FBF771FFEE2086
:10C50000FBF73EFFFBF7ACFF2046FBF739FFFBF7DD
:10C51000A7FF2846FBF734FFFBF7A2FFFBF77EFFE0
:10C520000A20FEF7F2FA70BDF0B5002510260527A7
:10C530009C463F070B46BE620C4C06E0595DE1602D
:10C54000A168C907FCD0E1686D1C8542F6DB0020BC
:10C5500007E06146095CE160A168C907FCD0E168B9
:10C56000401C9042F5D3BE610020F0BD0030014078
:10C570000000010203040005405C0000A05C040010
:10C58000C06C0800805C0400E03F1E00E07D1E00DF
:10C5900007A9022570889B880A0016000100060082
:10C5A0000100020087008D002D001A3152001A335D
:10C5B0009A001A351D011A376B003B31BE003B3320
:10C5C0005E013B3596023B37000099599959EB5172
:10C5D0008F421E45142E0080EB51F5283333E13A8B
:10C5E000703DE13AC235852BC2353333C235C23591
:10C5F000AE47E13A5138A330513800000000000046
:10C6000000000102030406070809030406080C10D1
:10C6100018203000000000010203040000000000A8
:10C62000000000000000F03F000000000000F83FA4
:10C6300000000000000000000000004003B8E23FDE
:10C64000000000000000000006D0CF43EBFD4C3E90
:10C65000033333333333E33FFFAB6FDBB66DDB3F85
:10C660004D268F515555D53F01411DA96074D13FCD
:10C6700065DBC9934A86CD3FEF4E454A287ECA3FC7
:10C680003E5555555555C53F93BDBE166CC166BF49
:10C690002CDE25AF6A56113FF16BD2C541BDBBBE42
:10C6A000D0A4BE726937663E0000000000000000A2
:10C6B000D0C6000800000020880100006C5B000864
:10C6C00030C7000888010020501A000068A8000840
:10C6D0000124130704380D091E0805400826091017
:10C6E0004008560A131D043B08BE0516D8BC40106E
:10C6F0000852010338C842035E5C121B0202C514D3
:10C700000901022281F01F66810498899686967934
:10C71000821598039814988796749778824397881F
:10C72000967197778249D90149294F920492200046
:04000005080050C1DE
:00000001FF
